:020000040800F2
:10000000703000202D2F0008DB980008192F000801
:1000100000000000000000000000000000000000E0
:10002000000000000000000000000000093000088F
:100030000000000000000000992F0008115D00087A
:1000400079310008793100087931000879310008E8
:1000500079310008793100087931000879310008D8
:1000600079310008793100087931000879310008C8
:1000700079310008793100087931000879310008B8
:1000800079310008793100087931000879310008A8
:100090007931000879310008793100087931000898
:1000A0007931000879310008793100087931000888
:0C00B0007931000879310008793100082E
:1000BC0002B4714649084900095649008E4402BCF5
:1000CC007047C04602B4714649084900095C4900B2
:1000DC008E4402BC7047C046002934D00123002254
:1000EC0010B488422CD301242407A14204D28142AB
:1000FC0002D209011B01F8E7E400A14204D28142BB
:10010C0002D249005B00F8E7884201D3401A1A4337
:10011C004C08A04202D3001B5C0822438C08A0426E
:10012C0002D3001B9C082243CC08A04202D3001B24
:10013C00DC082243002803D01B0901D00909E3E79E
:10014C00100010BC704701B5002000F05FF802BD34
:10015C000029F8D003B5FFF7C1FF0EBC4243891A42
:10016C001847C046002941D010B404004C40A446A6
:10017C0001230022002900D54942002800D5404225
:10018C0088422CD301242407A14204D2814202D2FA
:10019C0009011B01F8E7E400A14204D2814202D21A
:1001AC0049005B00F8E7884201D3401A1A434C0817
:1001BC00A04202D3001B5C0822438C08A04202D34D
:1001CC00001B9C082243CC08A04202D3001BDC0875
:1001DC002243002803D01B0901D00909E3E71000D2
:1001EC006446002C00D5404210BC704701B500207D
:1001FC0000F00CF802BDC0460029F7D003B5FFF79C
:10020C00B3FF0EBC4243891A1847C0467047C0461C
:10021C001C2101231B04984201D3000C10391B0A2A
:10022C00984201D3000A08391B09984201D30009EE
:10023C00043902A2105C40187047C0460403020245
:10024C0001010101000000000000000041420840D3
:10025C001C2101231B04984201D3000C10391B0AEA
:10026C00984201D3000A08391B09984201D30009AE
:10027C00043902A2105C401A7047C0461B1C1D1D9D
:10028C001E1E1E1E1F1F1F1F1F1F1F1F002B11D1E5
:10029C00002A0FD1002900D1002802D00021C94327
:1002AC00080007B4024802A14018029003BDC046E2
:1002BC005DFFFFFF03B4684601B5029800F039F802
:1002CC00019B9E4602B00CBC7047C046D0400B0050
:1002DC00D1409C46203AD340184352426346934047
:1002EC00184370479140030090409C46203A93403D
:1002FC00194352426346D3401943704710B5002945
:10030C0003D1FFF785FF203002E00800FFF780FFE4
:10031C0010BDC04603000A7801311A700133002A5F
:10032C00F9D170470023C25C0133002AFBD1581E5F
:10033C007047F0B506000F0015001C0085B08B420D
:10034C0063D801D1824260D821002800FFF7D6FF84
:10035C00390000903000FFF7D1FF009B21001B1AE1
:10036C001A0028000393FFF7BDFF00900191B942DA
:10037C0045D801D1B04242D8009B019C01200021FC
:10038C00039AF61AA741FFF7ADFF04000D00039B7B
:10039C00002B2BD0019B009ADB0750081843019BC4
:1003AC005908039B9C46B9422CD801D1B04229D89C
:1003BC0032003B00121A8B41012692185B41002738
:1003CC00B6185F4101235B429C446346002BEAD183
:1003DC0030003900039AFFF779FF039AA4197D4185
:1003EC0006000F00FFF77EFF241A8D410A9B002B9D
:1003FC0001D01E605F602000290005B0F0BD002414
:10040C000025C4E7B6197F41DCE700240025EDE7A1
:10041C0070B5294D03212800284A09F072F9284E9D
:10042C0030000AF035F8002808D1012128001324E7
:10043C00244A09F066F96442200070BD102031692D
:10044C00B3680A6882430A60A022042130001B684A
:10045C0012039847041E06DA1B4A230001212800C8
:10046C0009F056F9E8E700F02BF9041E01DA174AF7
:10047C00F3E700F08BFA041E01D0154AEDE700F00B
:10048C0031F8041E01DA134AE7E700F017FA041EEC
:10049C0001DA114AE1E703212800104A09F031F989
:1004AC00B36810215B693000984700F037F80021E1
:1004BC000B4807F03FFFF3E7A8AD000842B1000876
:1004CC0010AB000870B100088CB10008ADB1000889
:1004DC00D3B10008F7B100081CB2000840B2000804
:1004EC008813000010B5094809F0D2FF031E084814
:1004FC0006D10121074A09F004F91320404210BD2E
:10050C000321054A09F0FDF80020F8E750AB00087C
:10051C0070AD000866B200087FB20008F0B5A7B055
:10052C00444B03939B681B68002B07D00F2502AA32
:10053C00AD18290003989847041E01D027B0F0BDD0
:10054C003D4F2A783B680A2A01D00D2A68D1002B2E
:10055C00E6DD0022394E3A49F254300008320AF0F6
:10056C0060F906AD002808D10121080000F0EAF876
:10057C0034492800FFF7CEFE40E033490922300011
:10058C000AF04FF9011E04D1012000F0DBF82F49CD
:10059C00EFE7082230002E490AF043F9002805D174
:1005AC000121023000F0CEF82A49E2E72A4909225B
:1005BC0030000AF036F9011E04D1022000F0C2F816
:1005CC002649D6E70622300025490AF02AF90028E8
:1005DC001CD1013000F006F9224E002800D0224E2A
:1005EC00022000F0FFF81F4B002800D01E4B009398
:1005FC008021330028001D4A08F040FA2800FFF73C
:10060C0091FEA04204D800233B6089E71849B0E76B
:10061C00295D039B03989B6801345B689847EDE761
:10062C003E2B04DC591C39600449CA5478E73C6001
:10063C0076E7C04650AB00081008002014140020C8
:10064C0097B20008A0B20008ABB20008B5B200081F
:10065C00C1B20008CAB20008D5B20008DFB2000867
:10066C00EBB20008B1B200089DB20008F2B200086B
:10067C0009B300080300F7B519790068DB888268B4
:10068C0094460269DC0715D4B02464032343012784
:10069C003D000A4C16681C408D4001943400AC435C
:1006AC003B4201D034002C43634614601B68019A12
:1006BC009847FEBDD02464036340E8E7FFFFEFFFDB
:1006CC0070B5174809F0E4FE164D002808D1012139
:1006DC0028001324144A09F014F86442200070BD59
:1006EC00124809F0D5FE0028F1D01148FFF7C2FFDF
:1006FC00041E06DA0F4A23000121280009F008F82D
:10070C00ECE70D48FFF7B6FF041E01DA0B4AF2E7DF
:10071C00032128000A4A08F0F4FF0024DEE7C04653
:10072C0030AB0008B8AD00082EB3000810AB0008C1
:10073C0024AE00084AB300081CAE00086CB30008D5
:10074C008EB30008B0B50C0000AF012820D11B48B7
:10075C0008F027FC002819D1194B1C70194B002CE0
:10076C0000D0194B6C4688B06A46184993618023B7
:10077C009B009383164B51611361E62115480023AE
:10078C001032490101F038F80020A546BD46B0BD35
:10079C0002280FD1104808F004FC0028F6D10F4BAA
:1007AC001C70084B002C00D0074B6C4688B06A4676
:1007BC000B49DBE716204042E8E7C04624AE0008B0
:1007CC0055140020B1B200089DB20008A7B3000870
:1007DC0003000001B8AD00081CAE00085414002042
:1007EC00B0B300080300012802D1044B18787047FD
:1007FC000020022BFBD1024BF8E7C0465514002019
:10080C0054140020082390B587B000AF0C00F818E2
:10081C000021102209F0FDFF012321685B423B609F
:10082C0079606379DA0703D5802212060A437A606D
:10083C009A0704D580227968D2050A437A605A0750
:10084C0001D50122BA721B0703D50223BA7A1343CE
:10085C00BB7223793B7209F07CFF0A220023FFF75D
:10086C0015FD786123791A1C082B00D908220C235A
:10087C002100F818D2B2083109F0C2FF1821380053
:10088C0000F068F88AB0216823796A461362052360
:10089C000748D1615061074813619061A42100237E
:1008AC0005481032890100F0A7FFBD4607B090BD86
:1008BC00C6B3000852B4000888AD0008F0B587B084
:1008CC001C4F380009F0E4FD1B4E002809D1012112
:1008DC0030001324194A08F014FF6442200007B0BA
:1008EC00F0BD0A226846164909F08AFF69463800AD
:1008FC0009F0B9F8041E06DA124A2300012130006F
:10090C0008F006FFEAE70025012203AB1A72380053
:10091C002A000D4903955D6003F09AFA0400A84281
:10092C0001DA0A4AE9E703213000094A08F0E9FE36
:10093C002C00D3E770AB000888AD0008DFB30008CB
:10094C0010AE0008F4B300081108000811B4000838
:10095C0031B4000880B500AF88B06A46084BD1614D
:10096C005361084B842193610423136100230648CF
:10097C001032890100F040FFBD46002080BDC0460A
:10098C006DB40008F0B40008F0AD000870B50C4D63
:10099C00032128000B4A08F0B4FE002001F060FE91
:1009AC00041E07D001210300074A280008F0B0FEFE
:1009BC00200070BD03212800044A08F0A2FEF7E7CE
:1009CC00F0AD00088DB40008B7B40008D0B400082E
:1009DC00F0B597B0059304230B921A400B9B0A9227
:1009EC00DA0807231A40013207001C9D03910D926F
:1009FC00820700D0C5E1041D002804D0072909D8BE
:100A0C001C20404254E1039A1A401300A4180822F7
:100A1C00D31A0393059B0426013B069300230993E9
:100A2C000C9304930293013B07930196002F01D082
:100A3C00059B23600D9B002B00DDF1E09D4B059A7F
:100A4C009A4203D39C4B9A4200D2E9E00B99E21BE9
:100A5C009308890700D50DE1049A0F2A00D9BBE051
:100A6C00002F00D10EE104990EAA53540A000799E5
:100A7C0012AB99540C9B01330C93F4E008260196AD
:100A8C00069B01330693069B9878002800D105E15C
:100A9C00029B002B08D12528F2D1079B0133079329
:100AAC00012302930426EAE77A284AD84B280ED869
:100ABC00472846D829282CD825283FD041D820288B
:100ACC00DED0233843425841C3B20293D8E74C38A6
:100ADC002E2836D8FFF7ECFAD43535353535353583
:100AEC00353535353735353535353535356135377A
:100AFC0037616161D437D235D4351837183535792B
:100B0C00E63735353735E600002308930426029383
:100B1C0027E0012213002A38C0B2834067490B42F8
:100B2C00AED1E2211800890508400B4235D11900DD
:100B3C00114002911342A3D0089013E0079B013B94
:100B4C0007930023C1E70022069B08925B78029270
:100B5C006C2B07D10426069B01961B786C2B01D1BC
:100B6C00B6190196013CA0193100FFF7B5FA704394
:100B7C000400002F3BD0019B039ADB1B1B189342F4
:100B8C0000D93DE7089B002B41D1019B042B20D1C0
:100B9C0008CD03600423043415E0072107358D4389
:100BAC0064188C430CCD002F08D00131C91B03985D
:100BBC000919814200D923E72260636000230826CB
:100BCC0002933300083401935AE7029B08930023E5
:100BDC009CE7019B082B01D0162012E70723073551
:100BEC009D430CCD0260436008230834EBE7089B5F
:100BFC00002B0CD1019B042B01D10435CAE7019BBE
:100C0C00082BE9D10735013B9D430835ECE7069BE2
:100C1C00023306930D9B013B0D9308CD059305E71D
:100C2C000B9B9B0722D50121E21B9308802080009F
:100C3C008242D1D2049A0F2ACED8002F1CD004980D
:100C4C00DBB20EAA13549C46079B12AA135400291C
:100C5C0000D10FE780226346524213430EAA13546D
:100C6C00099B01330993049B01330493069B0434C1
:100C7C00013B07E70021D9E7002903D0039B01338F
:100C8C000393F0E7039B023303930A9B002BEAD1F7
:100C9C000598FFF747FB039B1B18F1E78022E31B2A
:100CAC00D200934298D2002F0AD103980838C0186A
:100CBC0017B0F0BD98A900085CC70008DAFF000067
:100CCC009B08302238603B706B469B180A9A1B7845
:100CDC00002A0BD0FB70099BBB70002B1BD100258D
:100CEC000EAE049BAB421BD1E01BE1E77B70F2E73D
:100CFC000EADED560EA9595C002D07DA039E1519A1
:100D0C000140B54200D97BE62170013401330499CE
:100D1C009942EDD1E3E7012200237F20D21BF6E7B5
:100D2C00099B002B02D033787F2B1BD80A9B002BFE
:100D3C001BD012ABEB5C2370002301340193012315
:100D4C00019ADB1B1B199B18039A934200D957E697
:100D5C003378019A237001342000059909F050FD75
:100D6C00019B1C1901350136BBE733789B00FB183E
:100D7C001A6805920A9A05981A60FFF7D3FA431C71
:100D8C00DCE70E203DE6C046F0B59BB000AF3B6201
:100D9C008023FB181B6806001B07DB0F7B61837825
:100DAC00F9623A63BB6300290AD10478BB6BA400D7
:100DBC00E41845780419FB6A9D421BD8A31BFB62FF
:100DCC00F378BB61BB6B002B04D08023FB181B6832
:100DDC00DB0719D4BB69002B47D13B6B002B03D02D
:100DEC0030003A6AF96A9847FB6AFB63BD46F86BB8
:100DFC001BB0F0BD01342000FFF794FAFB6A013000
:100E0C0001332418FB62D6E73378FB619B007B62CD
:100E1C007368BB627B6AF5183B6B002B00D029E131
:100E2C00FB6AFB63BB6BEC180023BB63A54232D09F
:100E3C002B789B009859FFF775FA84217B181B6857
:100E4C000130002B0CD08822BA18BB6B126893426D
:100E5C0006D27A1812685B009852BB6B0133BB63E5
:100E6C00FB6B01351B18FB63E0E78023FB181B6849
:100E7C009B07B2D53378FB619B007B627368BB62C6
:100E8C007B6AF5183B6B002B77D1FB6AFB63BB6B62
:100E9C00EC183B6BBB6380220523BA181268250043
:100EAC0013405A4253410133FB62BB695B00E318A8
:100EBC003B633B6BAB4299D02B787B636B789B008D
:100ECC009C59B84B9C4202D3B74B9C4223D37B69B1
:100EDC00002B33D0796BB86A08F014F900282DD0A8
:100EEC006C468AB06A46B14B5361BB6A93617B6BAB
:100EFC00D36180239B001384AD4B1361922100239B
:100F0C00AC481032890100F077FCA546FB6B023B24
:100F1C00FB630235CDE77B69002B05D0796BB86A92
:100F2C0008F0F0F80028DBD180230122FB181B68A5
:100F3C00134209D1FB6BFA6A9B1AE9E78023022260
:100F4C00FB181B681342E4D02000FFF7EBF9842157
:100F5C007B181B68002B0DD08822BA18BB6B12684B
:100F6C00934207D2791809685B00421C5A52BB6B3A
:100F7C000133BB63FB6B1B18CAE7BB6B1C1E7B638B
:100F8C0015D0802104237A1812681A4014007A6351
:100F9C007A1812681A420AD00023BC6B7B63183390
:100FAC0040229B182900BA6BD81909F029FCBB6B9D
:100FBC00EB18FB60FB63BB695B003B613A69FB6848
:100FCC00944663447B60FB6B7A68934257D17B6B8E
:100FDC00757800215A198023FB181B68D2B29B0725
:100FEC0000D461088020381800680023C00705D49D
:100FFC008033FB181B685B07DB1723407270B370E0
:10100C00F17030003A6A796A3B6B9847F8630028B4
:10101C0000DAEBE6FB6940203370BB6B2100B37048
:10102C00BB693A6AF37018231B18D81975703B6B9F
:10103C009847041E00DAB1E0FB6ABA6BF868991A9B
:10104C007B6A3A6AC91A3B699C46C91A60443B6B75
:10105C009847002800DAA3E00025FB6B1C19231825
:10106C00FB637B6B9D4261D300213A6A08003B6BAA
:10107C009847BBE6BB6B00247B63082390E7FB6BB4
:10108C00484A1B78BB60FB6B5D78AB009B59934265
:10109C0002D3454A93420CD37B69002B30D0B968FC
:1010AC00B86A08F02FF800282AD0FB6B0233FB63D8
:1010BC0089E77B69002B05D0B968B86A08F022F87B
:1010CC000028F2D180230122FB181B6813420AD09E
:1010DC007B6B9B18073240215218796BD219DBB20B
:1010EC0055547B63E1E78023FB181B685B07DCD559
:1010FC00182240215218631CD2191555DCB2D4E7C2
:10110C0080230222FB181B68134203D07B6B063230
:10111C000133E0E7402118225218B968631CD21938
:10112C001155DBB20234E4B2D554BEE74022082399
:10113C009B18DB19EB5C0732BA18137084229B00E6
:10114C009B59BB63BB181C68002C09D08823FB1867
:10115C001B6800249D4203D2BA1812686B00D45A43
:10116C0047230121F8183A6A3B6B9847002817DB94
:10117C00FB6B1B18FB63002C04D1B86BFFF7D2F888
:10118C00013084B221003A6AB86B3B6B9847002857
:10119C0006DBFB6B01351B18FB6362E7F86325E686
:1011AC00F86323E698A900085CC7000815B5000889
:1011BC000400000168AD0008014B18607047C04680
:1011CC0000000020F7B504000D001E00019207F08E
:1011DC00F1F8030009F0D0FB054F32003B500199A8
:1011EC002800A04709F0C8FB385801F0B3FEC046F0
:1011FC0008000000802102200A4B0905DA6B82B03E
:10120C000A43DA63DA6B0A4007490192019A4A6889
:10121C00824300204A60DA6B04490A40DA6302B068
:10122C007047C0460010024000580140FFFFFFF716
:10123C0080230D4A9B00116882B00B43012113607F
:10124C000A4B0B4A1A600B4B1A6C0A431A641B6C40
:10125C00094A0B400193019BC0231168DB000B432F
:10126C00136002B07047C0460020024030000020DE
:10127C000024F4000010024000000140F7B5050006
:10128C000600002D01D13000FEBD2800FEF7DEFF68
:10129C0001238340DA430E4F04019D433B19019314
:1012AC001B7B0092002BECD0E3591B69002B09D15E
:1012BC00009B3C191E40636804221968019808F0D1
:1012CC00E3F9DEE7381998470028DAD1F0E7C04691
:1012DC0000AE0008F0B5002289B00F490F4809F0A4
:1012EC003CFA0024002600270E20C0220C4D03904F
:1012FC000696079728000B4B0B4904940294019413
:10130C000094920006F07CFD0849280009F036F99B
:10131C00200009B0F0BDC0463D130008C8050020F0
:10132C00500100204116000870140020DDB50008A3
:10133C0010B5024806F06EFB10BDC046CC00002074
:10134C00F7B500901F48019108F07DF9061E35D0C5
:10135C0000252800FEBD237B002B11D02368DB6801
:10136C00002B01D02000984763689F7123681B698C
:10137C00002B1BD1636804222000196808F084F943
:10138C0001361034104B9C42E5D3009B002BE0D06F
:10139C00002DDDD02800FFF771FF019B0500002B0D
:1013AC00F6D00021642006F0C5FFF1E72000984735
:1013BC000028DFD03B00B3401D43E1E705000127C7
:1013CC00024CDFE72408002010AE000800AE000835
:1013DC00014B8000C058704740AE0008030010B5A8
:1013EC000800002B05D0044A136000F0ABFC002071
:1013FC0010BD16204042FBE70400002010B5054C40
:10140C002378002B02D1044806F004FB012323703F
:10141C0010BDC04656140020CC00002010B50400AE
:10142C00074808F010F9002C03D00121054809F0F9
:10143C00C6F9054809F09DF9044806F0EBFA10BD11
:10144C001C08002020080020C8050020CC0000202B
:10145C0010B50021014809F0BFF910BD1C0800208F
:10146C0070B5FFF7F5FF0500084C094B9C4200D303
:10147C0070BD63685B79002B06D023685B68002B1A
:10148C0002D02900200098471034EEE700AE000887
:10149C0010AE000810B5044C0449200007F063FF9F
:1014AC00034B1C6010BDC046680000202CAE000829
:1014BC00140800200023FA210C4A10B513700C4AB2
:1014CC00890013600B4A0C481360FFF787FFFFF786
:1014DC00E1FF0A4B0A4918008B4200D310BD1A1ABF
:1014EC005C681211013222711033F5E75714002099
:1014FC001C080020200800205D96000800AE0008A3
:10150C0010AE000810B5044C01000022002320008E
:10151C0007F04AFF10BDC0466800002010B5024815
:10152C0007F0DCFF10BDC0466800002010B5034B6F
:10153C000100186808F023F810BDC04614080020FC
:10154C0010B5024808F054F810BDC04668000020E1
:10155C0070B5204B1878002826D0FFF7DFFF1E4C03
:10156C00051E2CD11D4B1E4C1B68002B11DD09F0E8
:10157C00F0F80A220023FEF789FE22686368801ABD
:10158C009941002903D1FA239B00984201D9FFF716
:10159C0067FF22686368FA200021800012184B4113
:1015AC0022606360FFF7CCFF70BD63685B79002B32
:1015BC0004D02368290020001B6898471034094B7D
:1015CC009C42F2D32800FFF7B1FF0121064809F035
:1015DC00F6F8C7E75614002000AE00081C080020DF
:1015EC00C005002010AE00082008002070B50E4D7C
:1015FC00297800290CD10120FFF7A2FE0B4C0C4BD3
:10160C009C4206D3FFF7A4FF0028FBD101232B70CB
:10161C0070BD63685B79002B03D0236820009B6846
:10162C0098471034EBE7C0465714002000AE000872
:10163C0010AE0008F7B500210800FFF781FE041E6C
:10164C002DD0FA2700267F0009F096F91C4B1D4A75
:10165C001B581360002B06D01B4B1B68092B02DD9B
:10166C001A4806F0D7F900230093002C07D020006D
:10167C00FFF704FE041E02D101277F423E00FFF754
:10168C0067FF0190002808D1009B114D002B13D14E
:10169C000E483A00330006F0EFF9019BE4E701270E
:1016AC007F423E00D0E72B689B69002B03D00022C1
:1016BC002800110098471035064B9D42F3D3E7E7FD
:1016CC00080000001808002020080020CC00002092
:1016DC0000AE000810AE000813B5154807F0B3FFB4
:1016EC00144B1B78002B0AD0EFF3108472B6FFF763
:1016FC002FFF002C02D162B6BFF36F8F13BD0E4BC0
:10170C001B68002BFAD0002809D1002200230B48BB
:10171C000092019300230A4A07F05CF9EEE70928CE
:10172C00ECD1064809F025F8064806F073F9E5E710
:10173C00200800205714002018080020C80500209D
:10174C0010270000CC00002010B5064B04001B68CD
:10175C0098472100A060044807F0A4FEFFF7BCFFE7
:10176C0010BDC0460400002068000020044B054A50
:10177C0000209B1ADB08994201D2C9008858704797
:10178C0000AE000850AD0008F0B55E1C85B0B50089
:10179C0000902800072317309843033080080F006F
:1017AC000192FFF7AFFE02AB04000322581D00218B
:1017BC0009F02FF803AB1E70002C0BD0039B2100FB
:1017CC002361002314312A1F0198C058C8500433D8
:1017DC009A42F9D1E023BA015B001A406D02054B25
:1017EC002A431A4020000023009907F071FF05B02E
:1017FC00F0BDC046C0FF0F00F0B591B004AF3B6028
:10180C000B035B0D0D0078607A613B610C0D002BB6
:10181C0000D173E0BB60002604237E62BE62FE62D0
:10182C0002931833FB1801930A23182200930233F6
:10183C009B18DB193200B9687869FFF7A5FA802389
:10184C00F8601B01984224D37B696C461A795B794A
:10185C008AB01B0213437A69927912041A437B698A
:10186C00DB791B06134304AA9361294B2949D361E5
:10187C0080239B001384284B516113619221330008
:10188C00264810328901FFF7B7FFA546BD460DB0BB
:10189C00F0BDFB6817345B055A0D3A61204A1B0BEF
:1018AC0015401D43FB68E01807239843033080085C
:1018BC00FFF728FE041E15D0030010337B62FB6873
:1018CC00FE62BB62042302931833FB1801930A23B4
:1018DC001821009302335B18124AB9687869DB1936
:1018EC00FFF752FA3B690E4A5B0215401D432A0072
:1018FC0020003B68796807F0EBFEC7E72000072360
:10190C001730984303308008FFF7FCFD0400E9E72B
:10191C00FF070000F2B500080400000190AD0008BC
:10192C00FF01F0FFAB960008F0B587B00E9F0400E6
:10193C00150002910393002F15D00F9B10210593D6
:10194C00009300203B000D9AFFF742F8802306001D
:10195C001B01984208D30221174A1848184B07F06C
:10196C00D7FE07B0F0BD3E00072322000C9C1D40A3
:10197C001A40D2001734AD011543A0197202154359
:10198C0098430C9A0330120580081543FFF7BAFDF3
:10199C00041E09D0002F07D00F9B310000930D9A25
:1019AC003B001030FFF714F82A002000039B02992B
:1019BC0007F08EFED5E7C04631B6000890AD0008A2
:1019CC00FF0700004068002804D0044BC01AC00870
:1019DC0000B2704701204042FBE7C04650AD000802
:1019EC000EB417B5054C05AB04CB010020000193D8
:1019FC0001F0CCFB1EBC08BC03B01847799700085B
:101A0C0010B5CB0604D4890603D50349FFF7E8FFCC
:101A1C0010BD0249FAE7C046BFB20008BEB20008CA
:101A2C00F0B591B0079317AB1B7804000D0006922C
:101A3C000593002B00D1B4E002261B9B1B9A1E4081
:101A4C0001231A400C921B9A07331A4008921B9AD6
:101A5C00F8331A400992002707F014FE0200B8422E
:101A6C0004D020008D49FFF7BBFF0700002E09D0E2
:101A7C0044231B9A1A4235D12A0020008849FFF7CB
:101A8C00AFFF3F180C9B002B0AD0059A854B920098
:101A9C00D258002A00D1844A20008449FFF7A0FFC5
:101AAC00099B002B5AD0089B002B77D11D00069B5D
:101ABC00002B05D01A0020007D49FFF791FF05008F
:101ACC00189B7C48ED19002B00D0BEE01A9B002B14
:101ADC0074D11B9BDB0700D5DAE020001B99FFF7C4
:101AEC008FFFBEE00020744B1E688642C9D0734B3A
:101AFC0028001968FEF7F0FAFA253100FEF728FBEA
:101B0C00AD0069430A9008003100FEF721FB0E91ED
:101B1C00E1210D9009010A98FEF71AFB0B910B9825
:101B2C003C21FEF7D9FAE1210F9009010A98FEF742
:101B3C00D3FA0A900E9831006843FEF7CDFA0D9B4C
:101B4C0002903C210B980193FEF702FB20000091C0
:101B5C000F9B0A9A5A49FFF743FF92E7089B099D8E
:101B6C00002B08D0059A574B920020005649D258AA
:101B7C00FFF736FF0500069B002B05D01A0020004E
:101B8C004B49FFF72DFF2D18079B002B98D01A00FF
:101B9C0020004E49FFF724FF2D1891E700230793EF
:101BAC00E0E7079B4A48012B00D14248189B059D52
:101BBC00002B4AD11A9B002B53D000251A9F102FB3
:101BCC0000D9102720001B99FFF71AFF0026B542F9
:101BDC004CDC199B20001A783E49FFF701FF0126C7
:101BEC0007231E4203D120003B49FFF7F9FEB74201
:101BFC0042D9199B20009A5D3649FFF7F1FE013658
:101C0C00102EEDD1002620003449FFF7E9FE3300F9
:101C1C00199AD25C1300203B5E2B00D92E22200097
:101C2C002F49FFF7DDFE0136102E2AD007231E4266
:101C3C0003D120002849FFF7D3FE3300B742E7D881
:101C4C0020002549FFF7CCFEEDE7189B2200254923
:101C5C0007F024FA1A9B002BB0D1059B002B00D067
:101C6C0037E7200007F076FD11B0F0BD20001A49CF
:101C7C00FFF7B6FE0136AAE720001B49FFF7B0FEBE
:101C8C00BDE7199BDB1919931A9BDB1B1A93E2E72F
:101C9C002000054A0549FFF7A3FE1EE76EB60008B3
:101CAC0072B6000850AE000869B60008ADB3000863
:101CBC0097B60008799700082C0800202808002007
:101CCC007BB6000864AE00089BB60008A1B60008FD
:101CDC009F970008A6B60008AEB60008B0B600087C
:101CEC00B2B6000899310008ACB6000873B5114AB9
:101CFC0004000B000568914200D9130005216846C9
:101D0C000D4A06F0BBFE0600636828000B220B4947
:101D1C005B6807F010FD63683200280069465B6859
:101D2C0007F009FD636828001B2205495B6807F072
:101D3C0002FD73BD0F27000032BE0008D1B60008AB
:101D4C00B5B60008012310B500211C00074A9042CB
:101D5C0007D8074A002900D101231360054B1860EE
:101D6C0010BD210040085B00F1E7C04640420F0067
:101D7C00280800202C08002070B50D00040046181F
:101D8C00B44201D1280070BD217803480134836826
:101D9C005B689847F4E7C04650AB0008F7B5114BA9
:101DAC00114C5B6A0093114B0193019B9C4202D333
:101DBC008620404212E06368009DAB420FD3256938
:101DCC00002D0CD09F7803799C46664643791B0204
:101DDC003343FF2633409F4201D1A847FEBD243434
:101DEC00E3E7C046540800204B0100204B010020C3
:101DFC00F7B504000E001700144D154B9D4202D38D
:101E0C008620404218E0134B69685B6A99421BD3E9
:101E1C00AB69002B18D08A780192227994466046DF
:101E2C00627912020243FF2002400198904204D1D1
:101E3C003A00310020009847FEBD4A79012A03D1AF
:101E4C003A003100200098472435D6E74B0100209A
:101E5C004B01002054080020F8B505000E001700B7
:101E6C00094C0A4B9C4202D3862040420AE063692B
:101E7C00002B01D12434F4E73A00310028009847B4
:101E8C000028F7D1F8BDC0464B0100204B010020C3
:101E9C0010B508220021024808F0BBFC10BDC0465A
:101EAC000F09002030B50A4B0A4CA34201D3002085
:101EBC0030BD1A7F196AD2005218914201D12433D5
:101ECC00F3E708310D1F2D788542F6D10120EFE79D
:101EDC004B0100204B010020F7B56B460579DC1D4A
:101EEC000E0025706B0609D02800FFF7DBFF0028D9
:101EFC0017D00020124B1B78834212D0114F12487E
:101F0C00002E0FD02B000321104A07F0BBFC2078C9
:101F1C0001F0C2FCFB69002B02D02100082098477D
:101F2C000120FEBD2B000321094A07F0ABFC2078F1
:101F3C0001F0D4FCFB69002BF2D021000920EEE764
:101F4C000E09002054080020E8AD000817B700085F
:101F5C002AB7000810B5044C030020000121034AE5
:101F6C0007F090FC002010BDE8AD00083FB700085A
:101F7C0070B5050001F008FD0300040078330ED1A4
:101F8C002B0002210B4A0C4807F07CFC280007F0C0
:101F9C007DFC0A4A002413688343136007E0002881
:101FAC00F4D02B000121064A034807F06BFC2000FB
:101FBC0070BDC0465AB70008E8AD000818090020EB
:101FCC007BB7000810B5084C23785B069B0F0A33CF
:101FDC009B001B59181E05D02000044A0449984741
:101FEC00C043C00F10BDC046540800205C08002040
:101FFC0064080020F0B585B004000191042813D0CA
:10200C00012828D1204B1B78002B24D000F0F2FDA6
:10201C001E4E1F4B9E421BD20025336A0293337F08
:10202C00AB4204D82436F4E7FFF732FFEAE7029B11
:10203C00EF00DF19387901F0A7FC0390387907F02D
:10204C0025FC144A136883431360039B002B0FDA9F
:10205C0000220D4B1A700D4D0D4B9D420BD30E4BA8
:10206C001B6A002B02D020000199984705B0F0BDE7
:10207C000135EDB2D3E7EB68002B03D0210028002B
:10208C00019A98472435E7E70D0900204B01002001
:10209C004B010020180900205408002073B56B4632
:1020AC00040080781870637922791B0213436A4606
:1020BC0053800322E37813406A46137107F0E6FB62
:1020CC00234B06001B68234D03420DD0A47820003F
:1020DC0000F076FD2000FFF74BFF08F049FA0028CE
:1020EC0002D1963008F0DCFA684601F08BFB6B46A7
:1020FC0002001B7878321BD10221174A174807F0CF
:10210C00C1FB6B46187801F00FFC0300783318D133
:10211C006B4602211B78124A104807F0B3FB2B00C8
:10212C000120B933C43518702B6833432B6007E09A
:10213C000C4A0028E5D00948012107F0A3FB002038
:10214C0076BD0028EBD06B46074A1B78F3E7C046F8
:10215C0018090020540800209DB70008E8AD0008BD
:10216C00E4B70008C0B7000804B80008F0B5AE4FDB
:10217C000600BB690C00150085B0002B1FD131780F
:10218C00CB06DB0E012B00D1A5E0022B00D121E107
:10219C00002B2AD12A6870787F293BD9062813D0C6
:1021AC00082832D0002820D1012350701370C33777
:1021BC00397899400B4313700223236002E098474F
:1021CC000028DCD1002012E0F278B0781202104323
:1021DC00120A111FD6B2012907D9072A05D8C1B294
:1021EC000191796A0F78002F03D11620404205B077
:1021FC00F0BD4878B04204D10198984200D122E158
:10220C000133C919EEE70B78D7E7BA373B7813706F
:10221C000123D2E701380828E7D8FDF749FF48E643
:10222C0052E605E6E6E60B00B07801F06BFA002802
:10223C00C8D0DAE7F378B2781B027C6A134332D148
:10224C00FFF726FE3900B378BA310B70FB69002B0F
:10225C00B8D003209847B5E76378042B0CD0052B36
:10226C0014D0022B0AD1F378B27865791B02134390
:10227C009D4203D1012001E0E37801932378E41817
:10228C002378002BE8D10028AFD0D9E7F378B278C7
:10229C001B0213439D42F1D1019B002BEED1200078
:1022AC00FFF7FCFEEAE7FF2500200195E8E7F3784D
:1022BC00B2781B021343012B97D10022C3373A701B
:1022CC0080E7F378B2781B021343012B00D08CE724
:1022DC00C3373B7076E72B6802933B00BA331B780D
:1022EC00002B00D181E7737932791B021343DAB2E8
:1022FC0094467A6A01921578002D00D175E75078D2
:10230C000390022803D11079604500D9A4E052193A
:10231C00F1E7029B1A705A70039B4EE701998A18D9
:10232C000192A3E00B2A00D05FE70024FF25039461
:10233C0002950AE0019B5B78042B14D0052B2ED060
:10234C00019B019A1B78D3180193019B1B78002BDE
:10235C00F0D1FB69002B02D0072003999847002C81
:10236C0000D02FE741E7019BDB780293019B327988
:10237C009D7873791B0213439D42E1D1F378B278B7
:10238C001B021343029A9A42DAD1019B0024039355
:10239C00072DD5D87B19BB331A700134D0E773796C
:1023AC0032791B0213439D42CAD1B378029A9342ED
:1023BC000BD0019B9C78200000F002FC2000FFF762
:1023CC00D7FD43425841C4B2BAE70198FFF766FE05
:1023DC000400B5E773787F2919D9002B00D004E7E6
:1023EC0036792D6873060AD03000FFF75BFD0028A4
:1023FC0000D1FAE6BA373B78002B00D1F5E629007C
:10240C00300007F0B4FA00236B700233D5E6012BD1
:10241C000CD0032B00D0E8E6F378B2781B02134300
:10242C0000D0E2E6012107E054080020F178B378EF
:10243C000902194300D0D8E63000FFF74DFD002803
:10244C0000D0BFE6D1E62960022A00D0DBE6CB78CB
:10245C008A781B021343B0E672787F2900D861E7B3
:10246C00002A00D155E70A2A00D0BEE6019A12785C
:10247C00002A00D1B9E601994978042900D04DE72A
:10248C00019989788B4200D048E70022072B02D8AB
:10249C00FB18BB331A78029B1A70B9E6F7B5050026
:1024AC001F000426009101923B002800019A00991C
:1024BC0001F098FA030004000B330AD12B0002211F
:1024CC00054A064807F0DEF9013E05F0B7FE002E7E
:1024DC00EAD12000FEBDC04625B80008E8AD0008D2
:1024EC0013B5154C237D002B1ED1E26801AB802067
:1024FC00A1680192FFF7D2FF019AA3689B18A36011
:10250C00E3689B1AE3600ED1002A0CD02069E388A3
:10251C00834208DD2300C8331978FDF76DFE0029CE
:10252C0001D10123237513BD002180200B000A006B
:10253C00217501F057FAF6E754080020002330B556
:10254C0085B004000D000193984261D199423BD1B2
:10255C000B000822280002A907F018FA002804DA58
:10256C00802001F099F905B030BD6B462D4C029AD4
:10257C00DB892260039A257562602B4A2561A26073
:10258C006A46127AE56052B2002A10DB802B09D918
:10259C000121264A264807F0B4F8802001F07CF986
:1025AC002800DEE7002B02D02361E360DBE7FFF7B6
:1025BC0009FD0028D4D02269E388934200DD130082
:1025CC00E360FFF78DFFCEE7164D01ABEA68A96813
:1025DC00002A05DC020007F0D9F90028C3DABFE7AE
:1025EC0007F0D4F9002804DA802001F055F9200016
:1025FC00B7E7019AAB689B18AB60EB689B1AEB6072
:10260C00B1D1094BAB60FFF7DDFC0028D9D1A7E7AE
:10261C008028A8D1034BDA68002AD2D11B7D002B6D
:10262C00CFD1A0E7540800208C0800204CB800083B
:10263C00E8AD0008054B064A58629A62054A00202C
:10264C00DA62054A1A63054A9A61704754080020F9
:10265C0079210008A91D0008651E0008FD1D000851
:10266C00F0B5040085B04E4B009300980122524205
:10267C00D31705F00BF94B4B4B4D1B78002B0CD0A3
:10268C0002214A4A4A4807F03CF8782464420098F0
:10269C0005F074F9200005B0F0BD6B6A002B0DD16C
:1026AC0000F0CEF8FFF7C6FF6B6A002B06D10121B4
:1026BC00404A3F4807F025F80124E7E73E482C62E2
:1026CC00E8616E6A01F016F800F030FF041EDEDBE4
:1026DC0000F0B0FA041EDADB7378012B02D1F37927
:1026EC00002B06D10121354A314807F00AF816248F
:1026FC00CCE72A000026C832137002AA10005380BF
:10270C001671167001F07EF80400B042BFDB802712
:10271C0002AB18001F7001F075F80400B042B6DB74
:10272C00274B30001900019307F015F90400B04253
:10273C00ADDB3800019907F00EF90400B042A6DBBE
:10274C00204E214B9E4219D3002001F0EDF8041EBF
:10275C009DDB2E000127C436336880203B43336059
:10276C0001F0E2F8041E00DA91E7802332685B0284
:10277C001343B835002433602F7088E70024376A80
:10278C00337FA34201D82436DBE7E300FB1818792A
:10279C00196807F0E0F800288ED10134E4B2EFE7B5
:1027AC00B80000200C0900205408002065B800086F
:1027BC00E8AD000888B8000801200008ADB8000892
:1027CC00492500084B0100204B010020F0B58BB0CF
:1027DC001122194905A808F013F81022002101A8AC
:1027EC0008F017F8154C12220021200008F011F8FF
:1027FC00102101A802F0AEFE00281ADD082800DA2C
:10280C000820083801AB1B180F2021000022844639
:10281C0014276D46985CED190609AE5D6546284097
:10282C006D46ED19285C01320E7048700231082A91
:10283C00EED120000BB0F0BDE7B800085A14002010
:10284C00F0B58B4B8BB01B7800AF7B61002B03D0AA
:10285C008848BD460BB0F0BD864C874BBB6100234E
:10286C001D00FB603B61FB612378002B07D1834B80
:10287C0002349C42F1D101227D4B1A70E8E760785A
:10288C0005281FD8FDF71EFCAF03F1AF2153202202
:10289C007B69B9180B70402324217B847B697918E0
:1028AC000B70B81800F094FF002809D008237B8423
:1028BC001833F81800F08CFF002801D07B697B845A
:1028CC007B8CE3712378E418CEE7E378002BF9D105
:1028DC00A378002B21D03B690133DBB23B61F1E7DC
:1028EC006A6894421CD024359D42F9D36D4688B059
:1028FC006A46634B9461536103231361C221002325
:10290C00604810324901FEF777FFAD465D48012162
:10291C005D4A06F0F6FE00209BE75C4D5C4BE3E75E
:10292C00AB68002BD7D0200039699847D3E7002D2E
:10293C0057D1584A0121534806F0E3FEE6E7BB683D
:10294C002A6ADB00D3187B60A2781B799A423FD1AC
:10295C0001260322F3B23B60E37813402132BA180C
:10296C001370637922791B0213437B84A3787F2B2A
:10297C0024D93300012210339A401300BA691A4249
:10298C0023D180233A6813432022B91808000B7016
:10299C0000F01EFF002818D12023FB181B787A6842
:1029AC00A37013715BB2002B02DA3E681036F6B2DC
:1029BC000123B340BA691A43BA6183E70123B340D8
:1029CC00BA691A4201D1F3B2DEE70136102EC0D13A
:1029DC00BB680133BB602B7FBA689A42AFD32E4AD7
:1029EC00A8E70023F6E7FB68032B24D1FFF7EEFEE4
:1029FC00B860002812D0FDF795FC061E0ED01028EA
:102A0C0004D00221254A1F4806F07BFE3200A01C90
:102A1C00102E00DD1022B96807F0F2FE2378E218C0
:102A2C005B08E318911E121B032A0CD5FB680133BB
:102A3C00DBB2FB6046E7FB68002BEFD1FB69002B98
:102A4C0008D1174A76E77A69013B4A705A780A70BE
:102A5C000A00E7E7FB69FA69E31A93709BB21B0A59
:102A6C00D37013003A691A71E0E7FC612AE7C0469B
:102A7C0059140020DC000020010001004B01002053
:102A8C00F8B80008E0AD0008DEB900084B010020E2
:102A9C004B01002018B9000859B9000876B9000894
:102AAC00C1B90008094A0023110010B514788442FA
:102ABC0005D15468002C02D09B01C81810BD0133FD
:102ACC004032042BF2D10020F8E7C0462009002048
:102ADC00F0B504002C3C63680600257887B01033F1
:102AEC0027D1E16BE2688B0735D5002A07D1042387
:102AFC00194202D0002363601BE00B43E36305AB78
:102B0C002800A168FFF7CAFC031E08D00121294A3E
:102B1C002948009506F004FE16235B42EBE7059A64
:102B2C00A3689B18A360E3689B1AE36023699B1856
:102B3C002361636810330CD0236967690393A3691D
:102B4C00029307F015FD002828D031001B4807F030
:102B5C0003FD07B0F0BD05AB2800A16800F0AEFF87
:102B6C00031ED3D1059FA368DB19A360E368DB1BAD
:102B7C00E3602369DB192361002FBBD0280006F02A
:102B8C0014FF01003800FDF7E3FA0029B2D1E36825
:102B9C00002BAFD0280000F0D9FFCAE760613000ED
:102BAC00103804F037FF002FD3D02800029A039975
:102BBC00B847CEE70CBA0008F8AD0008F0060020C4
:102BCC0010B5EFF3108472B6FFF76CFF011E09D03D
:102BDC004368103306D18C235B4243602C3104488C
:102BEC0007F0BAFC002C02D162B6BFF36F8F10BD98
:102BFC00F006002070B500250C4CEFF3108672B671
:102C0C006368103307D18C2321005B420848636052
:102C1C002C3107F0A1FC002E02D162B6BFF36F8FEE
:102C2C0001354034042DE8D170BDC0462009002088
:102C3C00F006002070B500250126084C200008493C
:102C4C0007F072FC2000320031001038013507F01B
:102C5C0049FC4034042DF1D1002070BD4C090020FA
:102C6C00DD2A000810B5034A03480021121A06F0A9
:102C7C0020FE10BD70140020500100200648074AA9
:102C8C0010B5121A064906F018FE064A06480749FE
:102C9C00121A06F012FE10BD000000204B0100209D
:102CAC005CC7000800000020000000205CC7000882
:102CBC00F0B585B000AF0C1EB86036D06E468AB049
:102CCC006D4609686268A3682B6205232048A961D8
:102CDC006861EA612B61A1212A001E481032002391
:102CEC0089017A60F860FEF787FDB546E168AD466C
:102CFC00226963692B6205231748A9616861EA613F
:102D0C002B61A12100237A68F8688901FEF774FD14
:102D1C00B546E3690121114AF86806F0F9FCA3698C
:102D2C0001210F4AF86806F0F3FCBB68012B07D1B0
:102D3C00EFF305830B4A0748B968103B06F0E8FC33
:102D4C002100B86804F02CFCBD4605B0F0BDC046AF
:102D5C0036BA0008B0AD000865BA000894BA00088D
:102D6C00A3BA0008D1BA000830BFFDE7F7B50A4B8B
:102D7C000A4D0600EF18CC1B2A00200008490193CD
:102D8C0007F03EFD60190021019A07F042FD380062
:102D9C00083C74660830FEBD040000000000000012
:102DAC0010AE0008054B5A699B689A4205D08023E7
:102DBC00034A5B0551680B4353607047E0130020D6
:102DCC0000ED00E0F0B53E4B8BB05B6800AF7B6074
:102DDC00DB05DB0D04003B6062B6BFF36F8F394E31
:102DEC00130EFF2B08D1F33B1340082B3DD10121CF
:102DFC003000354A06F085FC00252C003B68032B7F
:102E0C0039D1324A0121300006F07BFCA369304AEB
:102E1C00934202D32F4A934205D32F4A934249D36C
:102E2C002E4A934246D2023B1A882D4B9A4241D1EC
:102E3C002368012130002B4A06F06AFC266808231F
:102E4C002022F818210007F0DBFC7B6A002D33D020
:102E5C00DA0502D1244A13437B6208233000F918A7
:102E6C00FFF726FFBD460BB0F0BD01251207C5D5F7
:102E7C000C000025C2E7F822796852001B4B114266
:102E8C0000D01B4B6A468AB07A606A4693613B68F5
:102E9C001849103BD36180239B001384164B51615E
:102EAC00136191210023300010328901FEF7A4FC3C
:102EBC007B689D460026C2E75B0A5B02CCE7C046F6
:102ECC0000ED00E0B0AD000812BB00083DBB0008EF
:102EDC00BC00000890A900080000002000000020A1
:102EEC0002DF000054BB0008FF010000E4BA000838
:102EFC00F9BA000870BB0008040000010821024A5E
:102F0C0053698B435361704700ED00E0EFF3088089
:102F1C00EFF3098101B57246FFF754FF01BDC046BE
:102F2C00094880F3088872B608480949401880F3AC
:102F3C000988EFF314800221084380F31488BFF34F
:102F4C006F8F06F0D0FC000070300020701700204E
:102F5C000008000010B50A4B9B6883420DD1EFF3BB
:102F6C000583002B09D08022064B520559680A4371
:102F7C005A605A6A04490A405A6205F021FA10BD97
:102F8C00E013002000ED00E0FF7FFFFF15498A6889
:102F9C0015481044EFF3098CF0C043464C46554697
:102FAC005E466746F8C072B6104F114E4A698A6089
:102FBC003E60104C141920680F4C2060906E00235A
:102FCC009366002800D162B6074C10191030F8C86F
:102FDC009846A146AA46B346BC462438F0C88CF3A2
:102FEC0009887047E01300203000000004ED00E079
:102FFC000000000864000000200A00200420714634
:10300C00014202D0EFF3098001D1EFF3088081690E
:10301C00023909780229FFD001B5724606F051FC3D
:10302C0001BDC04643B2000605D41F221A4001233D
:10303C009340014A1360704700E100E043B2000680
:10304C0009D41F221A4001239340034AD367BFF3CC
:10305C004F8FBFF36F8F704704E100E030B5FF2551
:10306C0003220B00290040B20240D20091409B0188
:10307C002B40C943934000280ADBC0240A4A80082D
:10308C0080008018A40002590A401343035130BD3C
:10309C000F2210400838054A800880008018C26949
:1030AC0011401943C161F2E700E100E000ED00E0DE
:1030BC00FF22044B9343044A9360BFF34F8FBFF33B
:1030CC006F8F70470000000800ED00E010B5203A4B
:1030DC001360029B01245360039B06499360049B7D
:1030EC00A143D36080235B04D3610023916102650B
:1030FC00836610BDD111000870B50B4B150098609C
:10310C00426E0A4B0E001A602C1C86F309880020B4
:10311C00034B9847201C002100220023014C204720
:10312C000F990008D1110008E0130020200A00209C
:10313C001022014B1A61704700ED00E0F0B5C0247D
:10314C0000220326FF25A40010002F003040C000F1
:10315C008740054993089B005B1819590132B94304
:10316C0019511F2AF0D1F0BD00E100E010B5EFF3CA
:10317C000583054A103BDB00D118496898588847ED
:10318C00FFF710FE10BDC04690AB0008F0B587B03D
:10319C0007000E0014000021102268461D0007F0E5
:1031AC0038FB6A4602239370054B2A0021006846BF
:1031BC0001930497059605F08BFC07B0F0BDC04653
:1031CC002999000810B5024B1B689847002010BDC8
:1031DC00240A0020034B044A1860022391780B4305
:1031EC0093707047240A002010000020072310B5AC
:1031FC000449054A99430548521A05F015FF002069
:10320C0010BDC0467754002000400220280A002040
:10321C00F8B50600002501277378AB4200D8F8BD3D
:10322C0034786419200000F0FDF800280ED020003E
:10323C0000F022F9074AE1008B58002B06D05218F7
:10324C001F2138000C40A040516898470135EDB261
:10325C00E2E7C046340A00200022052010B50C4CD1
:10326C00110020706070FFF7F9FE0022062011009B
:10327C00A070E070FFF7F2FE0C220721054807F062
:10328C00C8FA002207201100FFF7E8FE002010BD4D
:10329C00400000204400002010B50400FF20002C4A
:1032AC0005D02000FCF7B4FF1F23181AC0B2044B42
:1032BC001856044BDA6F1443DC67FFF7B3FE10BDEE
:1032CC004000002004180240024AD36F8343D367A6
:1032DC007047C04604180240020000B508000329DC
:1032EC000AD80E4BFCF7EEFE02090C131968914339
:1032FC00196059689143596000BD19681143F7E78B
:10330C00596811435960196891431960F4E71968B9
:10331C001143196059680A435A60EDE700180240DE
:10332C0070B5FF230D001400002804D0FCF770FFCB
:10333C001F231B1ADBB2094AD8008358AB4203D1B6
:10334C0011184968A14204D0002B04D11550121851
:10335C005460002070BD10204042FBE7340A00206E
:10336C00FF2310B5002804D0FCF752FF1F231B1AB3
:10337C00DBB20021024ADB009950D218516010BD1B
:10338C00340A0020C022C30452031340032210B598
:10339C000724800803431A401B0C9C4099400448A6
:1033AC0092001218106EA0430843106610BDC04660
:1033BC0000180240C022C3045203134003228008A9
:1033CC0003431A40044918329200505807221B0C30
:1033DC009A401040D84070470018024013B50E4C6C
:1033EC00200007F055F8002807D10C4801210C4AA1
:1033FC0006F087F9132040420AE0402300933F3B3C
:10340C000193A3681B68002B03D0694620009847E2
:10341C0016BD5820EFE7C04630AA000878AD00086A
:10342C0090BB00081F2201210240030008009040BD
:10343C0010B502003F2B05D90C480D4A06F068F96F
:10344C00002010BD0B481F2B0AD8C36813409A42AA
:10345C0004D001691140891A4B4259410800F0E728
:10346C00C36A13409A42F9D0016BF3E778AD0008B8
:10347C00AFBB0008001802401F22012102400300CC
:10348C00080010B590403F2B06D90848084A06F0B2
:10349C003FF91620404210BD064A1F2B03D8D060BE
:1034AC0010610020F7E7D0621063FAE778AD0008EE
:1034BC00AFBB0008001802400200802103008A43C1
:1034CC000020072A08DC5AB20448002A00DA044813
:1034DC0024228B435343C0187047C046980D0020DC
:1034EC00B80E002010B5024802F0AAFD10BDC0466F
:1034FC00B40A0020044B020010B51800034906F072
:10350C001DFA1620404210BDD8AD0008EFBB0008D4
:10351C00044B020010B51800034906F00FFA1620F0
:10352C00404210BDD8AD000808BC0008F7B55B4C94
:10353C00200006F0ADFF002807D15949594806F084
:10354C0004FA132464422000FEBDA568AB69002B6D
:10355C0005D15549534806F0F8F90524F2E7534EC6
:10356C0000223100200098470028F2D12B68002B54
:10357C0001D14F49EEE720004E4998470028F8D179
:10358C00EB68002B01D14C49E4E73100200001AA83
:10359C009847061EF7D1019A484B9A4205D04849E4
:1035AC00404806F0CBF98624CCE7464D464BE872F2
:1035BC002B6008232B71063BEB71FF33FF3331007B
:1035CC00424801AA2B8106F01DFD041E07DB019B5E
:1035DC0032001979186801F0DBFF041E05DA2200AD
:1035EC003B49304806F0AAF9ADE7280002F0D8FCB8
:1035FC003849021E0BD1280006F0D3FD3649021EB5
:10360C0005D1280006F0BAFD021E04D03349254826
:10361C0006F094F9A1E7B921402390270400012674
:10362C0089006B52043168542D497F006B52043170
:10363C0068542C496B508323DB00E81800193200C6
:10364C003100243406F04EFFBC42F4D10022082095
:10365C001100FFF703FD0820FFF7E4FC8020224B4C
:10366C004005D96B214A014211D1D96B0143D96371
:10367C00D96B01400191019980215068C900014327
:10368C005160DA6B1A490A40DA6300245BE7802345
:10369C005168DB000B435360F7E7C04630AA0008C3
:1036AC001ABC0008D8AD000839BC0008D4AE00081C
:1036BC005BBC0008CCAE000876BC0008006CDC02D9
:1036CC009ABC0008B40A0020005C0040ACAE0008B4
:1036DC00B6BC0008D4BC0008E8BC0008FCBC000860
:1036EC000404000024070000001002400070004099
:1036FC00FFFFFFEFB822024B920098507047C04674
:10370C00B40A002013B504000848210006F05DFD42
:10371C0003000020834208D00548009301212300B8
:10372C00044A05F0FDFF0520404216BDB40A0020F6
:10373C00D8AD000811BD0008130042B213B5040047
:10374C00002A0BDA802801D1002B0AD01148220064
:10375C00114906F0F3F81620404216BD402B00D953
:10376C0040238022210091430C4A0D48890189187D
:10377C000A18210006F08CFD030000208342ECD0D7
:10378C000448009301212300064A05F0C9FF0520D7
:10379C00E2E7C046D8AD000808BC000824050000CC
:1037AC00B40A002037BD000843B210B50C00002B42
:1037BC0001DB002902D1FFF7ABFE10BD034B01006A
:1037CC00180006F080FD20600020F6E7B40A002007
:1037DC0010B502790378002A02D107495A0604D1A0
:1037EC0078220020134205D00449054806F0ADF8B4
:1037FC000120404210BDC0465DBD00087CBD0008E4
:10380C00D8AD0008F7B50378040018000193FFF752
:10381C0053FE051E10D06188438822798B4229D231
:10382C0080201B4E1B4F00018446F359012A06D100
:10383C004800C01860450ED316204042FEBDC91882
:10384C008142F9D200223000019906F0B8FD62885D
:10385C006A80F3590CE0C9180904CB18300001999F
:10386C0006F0ADFD63885B006B806388F2595B00EA
:10387C009B18F35122796388012A01D15B009BB21A
:10388C002B802379032BD7D800202B71D6E7C04689
:10389C00B40A00202407000037B50400FFF70CFE23
:1038AC00051E13D021000A4806F02DFD00280AD071
:1038BC00084D0090230028000121074A05F030FF35
:1038CC000520404201E001236B713EBD1620F8E754
:1038DC00B40A0020D8AD0008A0BD000873B50600DE
:1038EC00FFF7EAFD041E16D04379002B11D03100EE
:1038FC000A4806F036FD051E09D00948330001219F
:10390C00084A009505F00CFF0520404202E060716A
:10391C00E060002076BD1620F7E7C046B40A002010
:10392C00D8AD0008C7BD000873B50400FFF7C4FD8F
:10393C00051E1FD0104E037902882100300006F0BE
:10394C0055FC00280AD00D4D0090230028000121C1
:10395C000B4A05F0E5FE052040420AE063B2002B5D
:10396C0007DD084BA101C91820002A888919FFF727
:10397C00E3FE76BD1620EFE7B40A0020D8AD0008B0
:10398C00EEBD00082405000037B50400FFF794FDD8
:10399C0000281BD00E4883681B69002B01D1002026
:1039AC003EBD0C4998470228F9D121000A4806F07F
:1039BC0049FC0028F3D0094D009023002800012178
:1039CC00074A05F0ADFE05204042E9E71620FBE76B
:1039DC0030AA0008CCAE0008B40A0020D8AD00080C
:1039EC0011BE0008F0B585B0040016001F0003914D
:1039FC00FFF762FD002802D063B2002B07DB220028
:103A0C0029492A4805F09AFF16256D4248E01430E2
:103A1C00029000220023029804F02EF8051E06D016
:103A2C002A002349214805F089FF0B25EDE706F014
:103A3C009FFD002802D10830FFF700FB802C02D13B
:103A4C00402E00D94026210033001A48039A06F074
:103A5C0042FC011E12D0184A009123000121134888
:103A6C0005F05EFE029803F0D5FF06F081FD0028FC
:103A7C0002D10830FFF7D6FA0525C6E7802C05D110
:103A8C00002E03D002002000FFF756FE06F070FD5A
:103A9C00002802D10820FFF7C5FA002F00D03E60A5
:103AAC00280005B0F0BDC04608BC0008D8AD000821
:103ABC0035BE0008B40A002053BE0008F7B5040058
:103ACC00009117000193FFF7F7FC1A49051E04D06B
:103ADC0063B2C668002B07DA17491848220005F0B4
:103AEC002DFF16204042FEBD009B002B18D0BE427D
:103AFC0000D93E00124BA101C9182B693200C9181C
:103B0C00104B0098C91806F07BFEEB689B1BEB6012
:103B1C002B699B192B61019B002B08D10020E2E73C
:103B2C00002FF8D00849054805F00FFFF3E7019B7B
:103B3C001E60F3E77ABE00088EBE0008D8AD000800
:103B4C0024050000B40A0020AFBE000810B5040024
:103B5C00FFF7B2FC002802D063B2002B03DA20007E
:103B6C00FFF7C8FC10BDC368002B01D00020F9E79B
:103B7C00034BA1010288C9182000FFF7DDFDF5E712
:103B8C00D80F002070B5114C00234022802120005A
:103B9C0006F02CFB0023402219002000902606F092
:103BAC0025FB002576008323DB00E0184019243523
:103BBC0003F030FFB542F6D1B8239B00E358002B3D
:103BCC0002D000210120984770BDC046B40A0020E5
:103BDC00B82210B5044B92009B58002B02D0002148
:103BEC000520984710BDC046B40A0020B82210B575
:103BFC00044B92009B58002B02D0002106209847C2
:103C0C0010BDC046B40A0020BC23082270B5104C6D
:103C1C000025104E9B00E25032000433E5500E4B51
:103C2C0003CB03C2BB239B00E358AB420ED029004D
:103C3C0028009847094BE25AAA4207D0063BE35C9E
:103C4C007F2B03D831002800FFF776FD70BDC046EE
:103C5C00B40A0020D80F0020500D0020A202000052
:103C6C00F0B591B0029316AB069204CB03911B886E
:103C7C0004920193029B5C889B880134E418029B9C
:103C8C00DB88E418002A00D1D4E0FA23019A9B00C7
:103C9C009A4200D3CEE083680FA99B6A984700280C
:103CAC0000D0C9E0019B002B0CD1644B049A9A42C2
:103CBC0040D8634B93429B414A229343614A9446BA
:103CCC00634401930F9B0499180061430D93FCF717
:103CDC0003FA069B1B89984200D21800049B05909E
:103CEC0043430C93584B0A93029B059A1B899342AE
:103CFC0022DA0A98039B039ADB8892885B08191CCA
:103D0C00934200D9111C039B8AB21980069B1B8815
:103D1C009A4206D9029B19880B1C914200D9131C9C
:103D2C009BB2039A1380484B984201D186204042A3
:103D3C0011B0F0BD454BC4E70C990D98FCF708FA8F
:103D4C000990002930D1029BFA219B8889000793A6
:103D5C00029B5B880B930B9A079B9C18069BA4B247
:103D6C009B880893069B5D886B469E8C019B5843F1
:103D7C00FCF7B2F9069B301ADA8880B21700904231
:103D8C0006D9029BDB881F1C834200D9071CBFB2DB
:103D9C00731EDB1B9BB29C420FD2029B361B013E57
:103DAC00DB88B7B2BB4212D2049A059B944601330E
:103DBC0005930C9B63440C9396E708994C19A4B299
:103DCC009C4217D9361B013EB7B2BA42ECD86308F5
:103DDC009D4206D26A46958D0B9A9A4200D91D1CBB
:103DEC00ADB2661B079BB6B2B34205D2E51A1E00F4
:103DFC00ADB204E01C00EAE7089BB342F6D8FA2304
:103E0C00601C9B0058430999FCF766F9019A030062
:103E1C00101A9A4200D2981A0A9B9842C4D2039B59
:103E2C00059A5D809E80DF801A81002800D161E7B1
:103E3C000A90B9E716207AE7052078E700350C00E0
:103E4C0020A107006B030000FFFFFF7FEE020000C4
:103E5C00F7B5846800AFA446002928D0002B26D0E3
:103E6C001C7A1E685D68E40725D58024A405A6424B
:103E7C0001D2A54229D31D21082316486A468EB0CB
:103E8C007A606A461362936280239B00124C1386FD
:103E9C00124B54619061D1615662D562136100235B
:103EAC000F4810491032FDF7A7FC7B689D46162081
:103EBC004042BD46FEBD80242401A64201D2A5424B
:103ECC0003D30B2103230848D8E76446A469A04711
:103EDC00EFE7C046CCBE00080BBF0008080000018D
:103EEC0050AD000840440000D5BE000873B5140066
:103EFC001D0082683032064E83683A33B44204D8CF
:103F0C0001950094FFF7ACFE76BD16204042FBE70E
:103F1C0040420F0073B514001D0082684832064EF3
:103F2C0083685233B44204D801950094FFF798FE8D
:103F3C0076BD16204042FBE700127A0037B5436885
:103F4C000D009B691B689847041E06D001212B00AD
:103F5C00034A0448009405F0E3FB20003EBDC04634
:103F6C0058BF000858AD000837B543680D009B6971
:103F7C005B689847041E06D001212B00034A0448B5
:103F8C00009405F0CDFB20003EBDC0467BBF000871
:103F9C0058AD0008F0B59BB003934368050002913F
:103FAC0001920021482208A8DF6906F032FC2800A3
:103FBC00019905AAFFF7C2FF002818D17F22059BA3
:103FCC00134214D03F2248241B0A1A405443029B2C
:103FDC0000921C19A4B206AA08232100280005F09F
:103FEC006BFD021E05D03C493C4805F07BFD1BB027
:103FFC00F0BD04AB9B7B1B071B0FDAB2944608AADF
:10400C00137104ABDB7A990603D502215079014375
:10401C00517106AA9279910604D5042108A8467913
:10402C0031434171D20604D5082208A948790243CC
:10403C004A715AB2002A04DA102208A948790243BC
:10404C004A7106A9CE7908AA7606760E5B061FD5AC
:10405C00069BDB00DB080893012351790B4353715A
:10406C0062461F4B9B5C402B2FD808AA52799207B3
:10407C0013D4002B11D003220333083493432800AC
:10408C000AAAA1B205F018FD021E06D01549ABE72D
:10409C004B88DB045B0D0893E2E708A94B79F6002B
:1040AC00DB0710D5BB689E1933687268002B01D0F2
:1040BC00280098472800009A0399FFF755FF00281D
:1040CC0000D174E793E77B68EDE70121064A0348CA
:1040DC0005F004FDEEE7C0469FBF000858AD000890
:1040EC0024C40008C6BF0008EBBF0008F7B50500E4
:1040FC00066901225242D3171036300005F0F9FC44
:10410C001821280001AAFFF719FF041E28D110233B
:10411C00019A18219A4328000192FFF725FF041EEB
:10412C001ED101F0BFFE1821070001AA2800FFF7DD
:10413C0005FF041E14D10822019B134210D001F07C
:10414C00B1FE0E4BC01B98420FD91022019B1821B7
:10415C001A4328000192FFF707FF041E00D10B3C05
:10416C00300005F0CAFC2000FEBD1821280001AA71
:10417C00FFF7E4FE0028DED00400F1E700A86100A0
:10418C0070B50469050023790E00002B25D110347D
:10419C0001225242D317200005F0ABFC7F21F3889B
:1041AC003288013B0B40FF21013A52061A43B38877
:1041BC000902013B1B020B401A4333890849013B9E
:1041CC001B040B4028001C211A43FFF7CDFE0500F1
:1041DC00200005F092FC280070BD10256D42FAE716
:1041EC000000FF01F0B5036987B001931B7905004E
:1041FC004768002B00D06AE0386800280ED083682E
:10420C00019A1B6811689847041E07D02200314997
:10421C00314805F067FC200007B0F0BD2E69012283
:10422C005242D3171036300005F063FC18212800D9
:10423C0005AAFFF783FE041E0ED0300005F05DFCCE
:10424C0025482200254905F04DFC38680028E2D0AD
:10425C0083685B689847DEE70123059A18219A4327
:10426C0028000592FFF780FE041EE6D106F071FAD5
:10427C00029003912800182105AAFFF75FFE041E87
:10428C00DBD10122059B134208D1300005F035FC2F
:10429C00002CD5D10123019A1371BCE706F059FA11
:1042AC00029A039B801A994100290DDC03D1FA2351
:1042BC009B00984208D81821280005AAFFF73EFE5B
:1042CC000028DED00400E0E70B246442DDE778240C
:1042DC006442A0E7FCBF000858AD000826C00008E7
:1042EC00F0B506000D00076985B0072907D92A002B
:1042FC002A492B4805F0F6FB8624644242E03B79C0
:10430C00002B48D13B0010330193019801225242FB
:10431C00D31705F0EEFB1821300002AAFFF70EFEB2
:10432C00041E2CD11021300003AAFFF707FE041E37
:10433C0025D18022029BE90727D51A43102302922C
:10434C00039A13430393029B20211A008A43A80764
:10435C0001D50A001A436B071AD5C0239B001A43D8
:10436C00182130000292FFF7FFFD041E07D1102127
:10437C003000039AFFF7F8FD041E00D13D60019850
:10438C0005F0BBFB200005B0F0BD93430293DAE7C8
:10439C00044B1A40E4E71024AFE7C04649C00008BC
:1043AC0058AD0008FFFCFFFFF7B5502101AA04002F
:1043BC004768FFF7C3FD002835D199260125019BDD
:1043CC001A00324033422ED050212000FFF7CCFD92
:1043DC00002828D1019B2B4205D0A823A422200021
:1043EC00F98EFFF7D7FD019BDB0605D5B823B42268
:1043FC002000398FFFF7CEFD019B1B0704D5290048
:10440C00094A0A4805F06AFB019B1B0604D52900E2
:10441C00074A064805F062FB5021200001AAFFF76D
:10442C008DFD0028CBD0F7BD62C0000858AD000848
:10443C0078C00008F0B5040003698BB002935021DA
:10444C00200006AAFFF77AFD002805D106995F4BDC
:10445C000A001A40194201D10BB0F0BD50212000C6
:10446C00FFF782FD0028F7D1E022069B920413424D
:10447C0037D026692000B36807AA0093F36803932A
:10448C006368DF6904ABDD1D290005F0DCFB002847
:10449C0027D12B780193009B002B05D02000039B88
:1044AC00079A0199009DA847019B032B19D1012262
:1044BC00D42120005242FFF757FD051E11D13B7B42
:1044CC009D4254D31821200008AAFFF737FD00287D
:1044DC0007D10123089A18219A4320000892FFF76C
:1044EC0043FD8022069B5201134222D06768FB6970
:1044FC00009323690193F421200007AAFFF71EFD06
:10450C00002816D13F23079D1D4212D01F232D0AD0
:10451C00B98F1D40EB00C91808AE320008232000EB
:10452C0089B205F0C9FA021E36D02949294805F08E
:10453C00D9FA069B1B0408D50121274A254805F00A
:10454C00CDFA0298243003F065FA069B9B0004D543
:10455C000121224A1F4805F0C1FA069B9B0300D497
:10456C006DE701211E4A1B4805F0B8FA67E73A6867
:10457C00E90052181368002B0CD0002010603A6828
:10458C00200052187221526849429847300024305A
:10459C0003F040FA013592E72A00F8212000F67961
:1045AC00FFF7E2FC051EC4D1009BF6001B689B19AB
:1045BC005A681E68039218600198243003F02AFA96
:1045CC0029002000039AB04795E7C0460090823B33
:1045DC008EC0000858AD0008B4C00008C9C000085F
:1045EC00E4C00008F0B58FB00993436807920693B6
:1045FC00039004910C79DF690669784A231C0F2C0F
:10460C0000D90F23DBB2D35C002108220CA8059340
:10461C0006F0FFF801214025049BAC465A7953085B
:10462C000B40900128405B01034308A8C37480230E
:10463C00D008313D084025405B4200012B43034329
:10464C0090080840400103436046834308A88375E3
:10465C000F2A06D96249634805F044FA862464425D
:10466C00B3E033685B0707D40C231A4204D05E4ACC
:10467C005C4805F033FAF1E7059B402B09D9402340
:10468C0001210093594A5748059B05F049F8162417
:10469C00E5E7520707D50F2C08D955492200514898
:1046AC0005F020FAF3E75349082CF7D83379002B9F
:1046BC0000D18DE0442103980BAAFFF73FFC041EA8
:1046CC0000D082E00B9B1B0600D583E03300243323
:1046DC000893079A099B089803F0CEF9041E00D0A2
:1046EC007AE0343601225242D3173000079605F097
:1046FC0000FA3B7BA34241DC0126764204990CAACA
:10470C00D671049B49791B68C9073FD50C9ADB000D
:10471C00520FDB08520713430C9348257543069B35
:10472C00ADB2D98F0398691889B208230CAA05F089
:10473C00C9F93149041E16D1049B5B799B072DD412
:10474C00059B002B2AD0032206990333C98F934370
:10475C000831049A69180398083289B205F0B2F945
:10476C00041E1BD0254922001E4805F0BBF90798F2
:10477C0005F0C3F9089803F04DF926E03A68E1001A
:10478C008A582600002AB9D00134B3E751881C4856
:10479C005B05DB0C01400B435380BEE73B68149A6E
:1047AC00F5005A513B68159A5B195A600122D021C9
:1047BC00B2400398FFF7D8FB041E03D000223B68DD
:1047CC005A51D4E7079805F098F920000FB0F0BDC6
:1047DC00732444E7722442E70B2440E724C4000806
:1047EC00FFC0000858AD000822C100084DC10008E8
:1047FC007DC100089FC10008C1C10008EBC10008C1
:10480C0003E0FFFFF0B587B0039242680291D769CD
:10481C0001921A682A4912040A40802100245B681C
:10482C0006695B0509065B0D0B431A4310360592AE
:10483C00050001225242D3173000009605F059F9B9
:10484C007B7BA3420ADC1C2502211E4A1E4805F074
:10485C0045F9009805F051F96D422DE07A68E600B3
:10486C00B258002A0DD00134EBE7009805F045F959
:10487C007B68029A25009A517B68039A9B195A60AF
:10488C001AE00123382004AAD17923400133814353
:10489C00DB000B43D371019AA300518E2800C91879
:1048AC0089B2042305AA05F00DF9051EDDD02A00F6
:1048BC000649054805F016F9280007B0F0BDC046BA
:1048CC000000FF073FC2000858AD000813C20008E3
:1048DC00F0B51D00436887B00291039201932A7AC8
:1048EC000400DE69012A06D93A493B4805F0FAF87A
:1048FC00862464426AE0002A43D004AB076905228F
:10490C000021D81C05F085FF2A68049BD2005B0FA0
:10491C00D2085B0713430493802380216A68002527
:10492C00D200D2081B061343059A89050A4013438B
:10493C0010370593380001225242D317009705F027
:10494C00D8F8B37B9D4209DB0221244A224805F0AA
:10495C00C5F8009805F0D1F81C24CAE7B268EF003E
:10496C00BA58002A14D00135ECE7009805F0C5F8C8
:10497C00B368029A2C00DA51B368039ADB195A60B7
:10498C0022E02B00039A0299FFF73CFF04001DE084
:10499C0001231F2104AAD2782B4001330A405B016A
:1049AC00134304AAD370019B2000998E0823C919C4
:1049BC0089B205F087F8041ED7D0220008490648B2
:1049CC0005F090F8002C01DB737BE418200007B095
:1049DC00F0BDC0465FC2000858AD000883C2000895
:1049EC0013C20008F7B5436805000C1EDE690769A1
:1049FC00019305DA22002049204805F073F8F7BD31
:104A0C00103701225242D317380005F072F8727B2E
:104A1C0094421ADBB37B1849A21A934228DD002179
:104A2C00B368D2009950B36828009B185960019B59
:104A3C00998E891889B2082205F04AF81049021E8D
:104A4C0016D1380005F059F8D9E700227368E10057
:104A5C005A507368A4005B185A60019B0432598E3B
:104A6C002800091989B205F033F8021EE9D005496E
:104A7C00024805F037F8E4E7A3C2000858AD000877
:104A8C00BEC20008EAC20008F8B50469456823797B
:104A9C000600EF69002B46D0FA220023920005F0A5
:104AAC0030F8002807D00121204A214805F016F8DB
:104ABC0005256D420CE0286800280BD083685B68E4
:104ACC009847051E06D02A001A49194805F00AF81D
:104ADC002800F8BD0025300005F0F6F825713B7B69
:104AEC009D420BD3103401225242D317200005F003
:104AFC0000F8200005F001F80025E9E73A68E90024
:104B0C0052181368002B0CD0002010603A6830004B
:104B1C00521873215268494298472000243002F001
:104B2C0079FF0135DBE77825C3E7C04616C30008DB
:104B3C0058AD000830C30008F0B589B04568066967
:104B4C0004000A22002102A8EF6905F062FE0A2285
:104B5C00002105A805F05DFE3000103005F0BBFC0F
:104B6C003000343005F0B7FC397B30000A002430BB
:104B7C0005F0B8FC286800280AD005F089FC00284C
:104B8C0006D101214F4A504804F0A8FF132013E02E
:104B9C002000FFF7ABFA4D4A002808D1FA22002377
:104BAC002000920004F0ADFF002808D0484A464887
:104BBC00012104F093FF0520404209B0F0BD200014
:104BCC0005F082F81821200001AAFFF7B7F9002898
:104BDC00F3D1019A3F4B18211A4020000192FFF7A4
:104BEC00C3F90028E9D11021200001AAFFF7A6F98A
:104BFC000028E2D11021019A20008A430192FFF78C
:104C0C00B3F90028D9D18021200001AAFFF796F929
:104C1C000028D2D12B22019B80211A432000019223
:104C2C00FFF7A2F90028C8D1EA682B8A200002A954
:104C3C00FFF75CF9284A1630B9D06A696B8A2000F4
:104C4C0005A9FFF767F9254A1630B0D0200002A954
:104C5C0004F009FF021E04D021491B4804F042FF56
:104C6C0094E705A9200004F010FF1E49021EF4D1A0
:104C7C001D4A542120000192FFF776F900289CD19F
:104C8C009922582120000192FFF76EF9002800D0DC
:104C9C0093E703225C2120000192FFF765F90028BD
:104CAC0000D08AE70122E021524220000192FFF756
:104CBC005BF9002800D080E701002A6C200004F08A
:104CCC0007FF7AE775C3000858AD00085BC30008FE
:104CDC0016C300085BFCFFFF8FC30008B1C30008BC
:104CEC00DDC30008FBC3000899908203D02843D091
:104CFC002BD8A82842D011D884281CD00300883B7C
:104D0C009BB21C2B20D801229A4026490A4212D170
:104D1C00082B35D01C2B17D1902015E0B82831D09A
:104D2C000BD8B42830D00FD803000422AC3B9343EB
:104D3C009BB2002B08D11C4806E0CC2826D003D807
:104D4C00BC28F8D0C828F6D07047E02820D007D867
:104D5C00D8281FD0DC281FD0D428F5D1D020F3E7D9
:104D6C00F4281BD004D8E4281AD0F028E3D0EBE7C1
:104D7C00F828E9D1E820E7E7CC20E5E79420E3E741
:104D8C008420E1E79C20DFE79820DDE7C820DBE703
:104D9C00DC20D9E7D420D7E7D820D5E7E420D3E727
:104DAC00E020D1E701001101FFFF000070B543685E
:104DBC0008005E6C0D001400FFF798FF1D4B984225
:104DCC0034D03368C0180368582D1FD019D804226A
:104DDC009543502D17D1FF22F820990192051140CF
:104DEC00C002DA00024011430122FE201A40114396
:104DFC0040019A00024011431C225B0013400B43FC
:104E0C0001E0802D0FD02360002070BD02211A001C
:104E1C000A400B4200D0D022DB0701D42260F3E71A
:104E2C000D231343EFE73F221340ECE7862040426B
:104E3C00EBE7C046FFFF000070B5436808005D6CEF
:104E4C000E001400FFF752FF1C4B984232D0582E24
:104E5C0021D019D804239E43502E17D1FF22F821BC
:104E6C00A309120413400902E2080A401343012269
:104E7C00FE2122401343C900A2080A4013430E220C
:104E8C00640814401C4301E0802E0FD02B68C0181E
:104E9C000460002070BDD02323405A1E93410D2284
:104EAC0022405C000123002AECD1EFE73F23234092
:104EBC00034CE7E786204042ECE7C046FFFF0000CA
:104ECC0000001C08F0B5436885B05B6C0500002140
:104EDC00586903AA009305F095F8041E07DB039BA1
:104EEC0000221979186800F053FB041E08DA344AC2
:104EFC0023000121334804F00BFC200005B0F0BD69
:104F0C006B685E6C304F380005F0C2FA002851D047
:104F1C00BB68F1680193B368012B13D9019B08316D
:104F2C009B69002B0BD0002238009847041E09DA2D
:104F3C000121264A234804F0E4FB254AD8E75824EB
:104F4C006442F5E7019BF1681B68002B35D03800F3
:104F5C009847041EF1DB337E002B06D0280004F0AA
:104F6C00B3FE337E1B4A5B081360280004F0ACFED2
:104F7C008021280003AAFEF7E1FF041EBDD1039B8C
:104F8C00154A80211A4328000392FEF7EDFF041EF8
:104F9C00B3D18022C02128005204FEF7E5FF041E85
:104FAC00ABD12800FFF7C8FD041EA6D1009B1B69DE
:104FBC009847A2E713246442BFE75824FBE7C04696
:104FCC003DC4000860AD000830AA00085BC40008AE
:104FDC0085C400080065004000001C0873B54368D8
:104FEC000C005E6C1A4D280005F052FA00282CD0EB
:104FFC00AB68B268F168DB68012A17D90831002B5D
:10500C0007D1144A1448012104F07BFB05204042CF
:10501C000BE0280001AA98470028F2DB0F4B0198FF
:10502C001A68002A0CD12060002076BD002B01D11B
:10503C000B4AE7E7280001AA98470028EEDAF7E7C1
:10504C0019684900FBF748F8EDE71320DFE7C04685
:10505C0030AA0008A6C4000860AD00080065004036
:10506C00D2C40008024B18684005C00F7047C046F8
:10507C00001002400B8813B50C481B051A0D1B18A9
:10508C001B0D0C2B0ED80A4C486813191A680243D6
:10509C0000201A600B881B051B0D1B191B68019344
:1050AC00019B16BD86204042FBE7C0460000C0FCB9
:1050BC00001002400B8809481B051A0D1B181B0D0C
:1050CC000C2B07D80020064B4968D3181A688A4362
:1050DC001A60704786204042FBE7C0460000C0FCC7
:1050EC000010024070B508881F4B00050D0014001D
:1050FC001B68000D0C2818D8002801D1863870BD0B
:10510C0002380A2809D8FAF7DDFF260622242626BB
:10511C0008081D1D1D00FA23DB018022236029686D
:10512C005201914219D20020E9E7104A801800057B
:10513C00000D0C2803D80E4AC240D207EDD48620AD
:10514C004042DCE700F02AF9C3005B08E5E7094BB5
:10515C00E3E7094BE1E70023DFE7090B1800013116
:10516C00FAF7BAFF2060DEE730000020CC0F000019
:10517C00111100000024F400006CDC020C2806D88D
:10518C00044BC3400020DB0700D4863870478620D0
:10519C004042FBE73A1F000070B508880C00000580
:1051AC00000DFFF7EBFF00281EDB6368FF2B1AD006
:1051BC0001225802800F013082401F2099B21B0C33
:1051CC000340013A9A40094E89190D6895430D60C8
:1051DC00636899B21A0E1B0C03409A40130089198C
:1051EC000C6823430B60002070BDC04600100240C9
:1051FC000B880A4A1B05180D9B1810B51B0D0C2BA0
:10520C0008D8074BC0180368486898434342584174
:10521C00013010BDFFF7B2FFF8E7C0460000C0FC3C
:10522C0000100240F7B5524F00F0D0F8380004F0EF
:10523C00A7FD00F049FE1F214E4C4F4AA3683D00CC
:10524C001B051B0F9B009B580B40D840136801900B
:10525C000B401D41A84202D2280002F069F9FFF769
:10526C0001FF012808D0802322685B0013432360D0
:10527C00FFF7F8FE0128FBD12368404A1340236056
:10528C000123226E134323660223226E1A42FCD0A2
:10529C0080232268DB031343236080231B042268D2
:1052AC001A42FCD03822A3681340102B18D1FFF7F8
:1052BC00D9FE012808D0802322685B0013432360A9
:1052CC00FFF7D0FE0128FBD10722A3689343A3600C
:1052DC003823A2681A42FCD1A368294A1340A36060
:1052EC002368284A134080222360920423681342C7
:1052FC00FCD1254B2549186880260840802189025D
:10530C00014319608021186849020143196019682A
:10531C001F48760401400A431A601A6832431A6027
:10532C0000F040F823681E43802326609B0422680B
:10533C001A42FCD0A368124A1340A3600723A26848
:10534C009A43053B13433822A360A3681340102BE8
:10535C00FBD1019BAB4202D3280002F0E9F80D4BC4
:10536C000D4A1F60A36800201340A360FEBDC04619
:10537C000090D00300100240C4B00008FFC7FFFF2C
:10538C00FFF0FFFFFFFFFFFE0C100240FFFFC1FF0D
:10539C00FFFFFFF130000020FF8FFFFF0048704738
:1053AC000024F400064B074AD9681140064A0A4308
:1053BC00DA608022D96852050A43DA607047C04629
:1053CC00001002408C80FF1F0208002080210F4B30
:1053DC004905DA6B82B00A43DA63DA6B0A40802142
:1053EC000192019ADA6B49020A43DA634022DB6BC1
:1053FC000B400093009B064B19680A431A6020224D
:10540C0019680A431A6002B07047C0460010024087
:10541C00006C004010B5084805F03AF8002808D098
:10542C00064C2000FDF7D6FE2000FBF7C5FE002041
:10543C0010BD13204042FBE750AB00084D54000850
:10544C0070B50400074D0A2804D1AB680D21280063
:10545C005B689847AB6828005B68E1B2984720000E
:10546C0070BDC04650AB0008F7B547681E00036915
:10547C00B868009201930C0004F05BFA8023009A48
:10548C0005009B039A4215D12000BD68FDF792FFE1
:10549C0085420DD12100280004F04BFA0400FDF7E1
:1054AC0013FF2000FDF75CFF00212000FDF714FF27
:1054BC000020FEBD8023009ADB039A4224D0802377
:1054CC00DB049E421CD0C023DB049E421AD08023F6
:1054DC0016209B049E4218D1022628000D49019AE1
:1054EC00FDF71EFF002812D12000B968FDF74AFF16
:1054FC0028003100FDF7F0FE2800FDF7CDFED7E7C0
:10550C000126EAE70326E8E786204042D1E710208F
:10551C00FBE7C046B59F000870B5036904005860EE
:10552C000B4D280004F0B4FF00280FD0AB68616865
:10553C001B680C31002B04D028009847002803DC92
:10554C0070BD58204042FBE70020F9E71320F9E733
:10555C0030AA00081FB50B4B0C001B681BBA01933B
:10556C00094B1B681BBA0293084B1B681BBA0393AD
:10557C000C2900D90C24220001A905F041F92000C6
:10558C0004B010BD9875FF1F9475FF1F9075FF1F19
:10559C00F7B504000025C90043180193019B9C42F8
:1055AC0001D1002035E01F271023226817401A4232
:1055BC0017D1202563681D43F821530949000B407E
:1055CC00E2395209FF390A401A4300921B09192B80
:1055DC0020D8114A9B009E58002E0AD1132040421D
:1055EC0017E0102F03D0112FE6D16568E4E73025C2
:1055FC00E2E7300004F04CFF0028EFD00F230099B5
:10560C002A00194030003B0004F0E7FC0834002865
:10561C00C4DAFEBD1620E2E70CB0000870B50369D1
:10562C00C0225B680C001B68D2000B6080214368B1
:10563C0005001B68C9001B68134002228B4204D072
:10564C001C4A9B185A425341DAB2C0218020227165
:10565C006B6889011B6800225B6840010B40834228
:10566C0006D002328B4203D0013A002B00D002321A
:10567C0062716B681B6818681968C023DB001940DD
:10568C000D4B184004F008FDC022A0716B6892000D
:10569C001B689B681340094A9B185A425341DBB262
:1056AC00E3716A6812689268520400D503230020E3
:1056BC00E37170BD00FAFFFF0010001000FDFFFF4A
:1056CC00F0B5436885B000AF05001E6802697960CB
:1056DC00002939D01068D9688368DB68002B0DD09D
:1056EC000C22BA189847041E0BDA01211A4A1B48DF
:1056FC0004F007F82000BD4605B0F0BD5824644204
:10570C00F3E73368164A7968134033607B685808AE
:10571C00FB68C018FAF7E0FC0F2818D86C468AB062
:10572C002B686A4693617B680E49D36180239B008A
:10573C0013840D4B516113619121002307481032E2
:10574C008901FCF759F8A54616246442D2E780B2C9
:10575C000024F060CEE7C04689C50008D0AD000833
:10576C00FF7FFFFFB7C5000804000001F7B50C0070
:10577C00036941685D682379012B13D09A1E564248
:10578C007241920200926679022E0ED8494F760031
:10579C00F75BA679022E0BD0042E34D05E1EB341DB
:1057AC001B0308E0C022D200ECE78027BF01F0E722
:1057BC005E4273411B07E67901960026B446019EB2
:1057CC00012E02D1C026B600B4460968A5421DD1EF
:1057DC000C68394E009A3440224313430B604B68DB
:1057EC00364A13403B434B60436835491A6893680B
:1057FC000B4061460B4393602968FFF761FF00285B
:10580C0000DD0020FEBD80235B01D4E7C0220E68C2
:10581C00D2001640009AB24205D00E68294A1640B2
:10582C00009A16430E60C0264268B60111684A6899
:10583C003240974204D04A68204E32403A434A6084
:10584C004268214E11680A683240934204D00A68BB
:10585C001E4E324013430B60C021436889001A6806
:10586C0093680B409C4505D0936815490B406146E5
:10587C000B43936080224368D2011B6899681142E4
:10588C0006D0019A032A09D09A6811490A4004E00B
:10589C000199032902D199680A439A6021682B68FF
:1058AC009942AED0FFF70CFF0028ABDB23682B60CE
:1058BC00A7E7C0463CB10008FFE9FFEFFFCFFFFFB1
:1058CC00FFFCFFFFFFF9FFFF00100010FFEFFFEFE1
:1058DC00FFBFFFFFF0B5060045680469744885B04A
:1058EC0000AF206004F0D4FD002806D1714A0121DC
:1058FC00714803F006FF13240BE02068E968836805
:10590C001B68002B07D101216C4A6B4803F0F9FE90
:10591C00582464420AE09847041E0BD10C23002142
:10592C00286AFA1804F06EFB041E0BDA2000BD4640
:10593C0005B0F0BD0121614A5F4803F0E2FE002C86
:10594C00F4DBEBE7FB68002219791868FFF720FEFF
:10595C00041EEBDB0122756833692C685B687B6085
:10596C00236893432360686804F092FD002801D1FA
:10597C00534ABCE76868A9688368DB68002B00D0D1
:10598C009847EFF31082012383F310880C212368CE
:10599C000B43236082F3108830007968FFF7E6FE32
:1059AC00002801DA1624B4E72B7D002B03D0082342
:1059BC00A2681343A3606B7D002B04D08022636824
:1059CC00120213436360AB7D002B04D0802263680A
:1059DC00520213436360EB7D002B04D0802263687A
:1059EC009202134363602B7E002B49D0354B9C42B3
:1059FC0029D0354B9C4226D0344B9C4223D0344B7F
:105A0C009C4220D0334B9C421DD0334B9C421AD02D
:105A1C00324B9C4217D0324B9C4214D06C4688B00F
:105A2C006A463368936180239B002E4993832E4BE7
:105A3C0051611361E22100231F4810324901FBF729
:105A4C00DBFEA546AEE773681A6880239168DB011C
:105A5C000B43936022686B7E24495B050A40134319
:105A6C0023602268AB7E22491B040A401343236047
:105A7C00EB7E002B04D08022A36812021343A36098
:105A8C002B7F002B04D0802322689B0513432360BB
:105A9C00012322681343236080239B03E2691A428B
:105AAC00FCD08023DB03E2691A42FCD000243DE7E2
:105ABC0030AA00081ABC0008D0AD0008CEC50008FA
:105ACC00EEC500080038014000440040004800408A
:105ADC00004C004000500040003C01400080004061
:105AEC000084004009C6000803000001FFFF1FFCF2
:105AFC00FFFFE0FFF7B5436800901C6803690D00D9
:105B0C005B6801934B790A799C468879012A16D1F6
:105B1C00022B2ED9C02180230600C9009B0102282C
:105B2C0000D188E0042836D00020824237D0802073
:105B3C00033A4001012A32D886204042FEBD022A97
:105B4C0009D1022B23D980210600C900022860D07C
:105B5C0080239B01E6E7022B1BD9060000210228BB
:105B6C00F6D10021002A54D18020110040050322D7
:105B7C001AE0C021C9006646344B7600F35A060081
:105B8C000228CFD1002A56D18020400507E0802181
:105B9C00F0E70021EFE7002ACED1802040018027DA
:105BAC0000227F01BB423CD16245C5D104F074FA9E
:105BBC00B042C1D1EB79002B19D0012B42D1244B2F
:105BCC009C4214D0234B9C4211D0234B9C420ED0B0
:105BDC00224B9C420BD0224B9C4208D0214B9C4226
:105BEC0005D0214B9C4202D0204B9C42A4D10126D3
:105BFC0023682900B34300982360FFF7B7FD002802
:105C0C009ADB236800201E43019B266006CD06C349
:105C1C0094E7033A012A00D88EE78023002002265D
:105C2C009B01C0270222BF01BB42BDD0013A002B11
:105C3C00BAD00232B8E7033A012A00D87CE7022630
:105C4C000020ACE7032BBAD076E7C0463CB1000885
:105C5C00003801400044004000480040004C004027
:105C6C0000500040003C0140008000400084004097
:105C7C0070B580251049114B8C681B680E68104854
:105C8C008A686D02002C08D1002A11D11A002E420C
:105C9C0009D100681818801A70BD002A0AD02E424B
:105CAC0001D1A242F5D90468E41804600968F0E750
:105CBC001C00F4E71A00F2E710E000E0DC1300200F
:105CCC00D81300200A4A0020136A1B021B0A136215
:105CDC00C822084B52011A60074B084A1860084B3F
:105CEC005A600722986019680A431A607047C046C8
:105CFC0000ED00E0DC130020D8130020FF1800009A
:105D0C0010E000E0F8B50024FFF7B2FF104E2300BE
:105D1C003168104D0A00286869688018594128605C
:105D2C006960C8210C4D346049012E686F68801B76
:105D3C00FAF7D2F9C8214901414323000A0092190C
:105D4C007B412A606B6002F041FDFDF72BF8F8BD3A
:105D5C00D81300200806002000060020F0B53B4BAD
:105D6C003B4D87B0002960D0421C08D101212A6824
:105D7C008A432A60FF2212061A6007B0F0BD1B6826
:105D8C00039300230293012854DCEFF31083059353
:105D9C0072B6FFF76DFF00221100AB6804932D4B18
:105DAC001E685F6836184F41300039001860596022
:105DBC00294B009601971A60284B1C68009B1B1BF3
:105DCC0093423EDBC82702987F017843244A39006E
:105DDC008018C018FAF780F9009B7843E41A8023E6
:105DEC002018DB00984200D218001E4B984200D9B4
:105DFC001800164B174918600138AB686860002012
:105E0C00A860049AD41A9A421ED2039D6219030008
:105E1C000C684D6812196B410A604B60059B002B96
:105E2C00ABD162B6BFF36F8FA7E71B680393431C1C
:105E3C00A7D10D480D4B984200DD1800431E02936C
:105E4C00A3E78020C000D4E72200E0E7DC130020A9
:105E5C0010E000E008060020D81300200006002007
:105E6C00FF18000000DCFF003C0A00003D0A0000A7
:105E7C0070B5EFF3108572B6084A094B14681B68AD
:105E8C00E41AFFF7F5FE0019002D02D162B6BFF33C
:105E9C006F8FC8214901FAF71FF970BD0806002061
:105EAC000006002070B5EFF3108572B6054B1C6828
:105EBC00FFF7DEFE2018002D02D162B6BFF36F8F04
:105ECC0070BDC04608060020382370B51D4CA26872
:105EDC001A4205D123681C489B045B0FD84070BD47
:105EEC00A2681A40082A27D0A2681A40102A17D193
:105EFC00E368E168DB43E5684906490F6F322D0A18
:105F0C00013115409B0709D11048FAF7E5F8E16813
:105F1C006843490F0131FAF7DFF8E0E70A48F4E784
:105F2C00A2681A40202A09D0A26800201340182B1E
:105F3C00D5D1FA20C001D2E70448D0E78020000276
:105F4C00CDE7C046001002400024F40000127A0095
:105F5C000A2382B00193019B002B07D1054BC00093
:105F6C00C01800688001800D02B07047019B013B96
:105F7C00F0E7C046009800400A2382B00193019BD1
:105F8C00002B07D1054BC000C01840688001800D64
:105F9C0002B07047019B013BF0E7C04600980040FF
:105FAC0073B504000120002C2FD0244D635DDAB2B0
:105FBC00002B05D1A5239B002000E25404F0DDF852
:105FCC0003236355206800F02FFD002322001900E5
:105FDC00012620791432984218D1002122000800A1
:105FEC005532FF328B421BD16B46227C1A70E36810
:105FFC006168A268206804F00EFA00236374013310
:10600C006355237B012B15D0002076BD1370013313
:10601C005670D170116151619161DBB22832DAE7AF
:10602C00117001315070D070106150619061C9B223
:10603C002832D7E7200004F0DAF9E5E795020000F2
:10604C00F0B5040087B0006804F007FACA4B1A6870
:10605C0004231A420ED0802580222D021202054004
:10606C00104201D100F032FC8022256812026B6CC8
:10607C00134201D107B0F0BD0F270F226B6C1F40EC
:10608C00134200D0A4E0190001321140134221D177
:10609C002B68BA4A200013408022120213432B6053
:1060AC00237DB74ADB009B181B68A26A9B019B0DE2
:1060BC002363D318A36203F097FC637C002BD3D02B
:1060CC00E26A2168002ACFD18020637C0343CB6431
:1060DC006274C9E72B6880221E001201164013421D
:1060EC001BD0AA235B00E05CFFF746FF2200A72130
:1060FC005532FF3289000300D06161182800D28824
:10610C0001F0E8F921689F4B0A6820001A408023AF
:10611C0013430B60FDF778FDA6E71B04A4D52A6892
:10612C00984B1A40802313432B60AA2325005B0055
:10613C00E05C2768FFF720FF5535FF35031EE8614B
:10614C000ED0696900290BD03800EA8801F0C2F939
:10615C006B69EA6931009B1820006B6103F02FFC1E
:10616C0023681B681A0500D57EE7C02292011340F4
:10617C00934200D178E7824A53689B019B09536094
:10618C002B693E2B17D91F20590903405842434114
:10619C00C91A53688906194380231B060B435360A5
:1061AC002168794A0B681340C02292015A40774B00
:1061BC0013430B6058E7002B01D15168ECE7012029
:1061CC0059080340C9185368890619435160E7E719
:1061DC00BB00ED1801932B6803936B469B890293CC
:1061EC00039B1B043ED52A68664B1A40802313433D
:1061FC002B6028257D4365192B006133FF331A78FA
:10620C00236804932B005533FF33002A69D1187887
:10621C00FFF7B2FE0190002809D02B005B33FF334F
:10622C00FC351A88E96E0300049801F053F9282311
:10623C00190079436218FC32506F019D4019506768
:10624C00D06E4019D066106F002803D0926E954224
:10625C0000D3FDE07B43E3185533FF33200019785E
:10626C0003F0ADFB039B22681B0600D4FCE6BB00CD
:10627C00D218136841490B40802109020B4313606B
:10628C002823190079436618F27D012A00D018E101
:10629C007A1C53430022E3185A60731CDB7F934231
:1062AC0017D0039B5B0600D4E8E0737D934200D0CB
:1062BC00D5E0337D3249DB005B181A6892019209F4
:1062CC001A608022337D1206DB005B1819680A43C2
:1062DC001A6028237B43E318197D200003F084FB0C
:1062EC00C2E62A005832FF3212781E78022A00D0F9
:1062FC0086E08023029ADB011A400592029A300054
:10630C00FC351A4248D0FFF723FE2A6F0300019098
:10631C00824222D3121A2A6721D0029A52060ED533
:10632C0028227A43A2185532FF321178226889004C
:10633C005218106816490840164901431160002B89
:10634C0000D174E72821794361180A005D32FF32CD
:10635C00FC311288C96E206867E700222A67049A0C
:10636C00B6009619326808490A40802189015140CB
:10637C00064A0A433260D0E7A00001400F8FFF07A6
:10638C00009800408F0FFF078FBFFF078080000031
:10639C008F8FFF07C0800000FFF7EEFD2A6F030010
:1063AC00019082421DD3121A2A671CD0029A5206FF
:1063BC000ED428227A43A2185532FF321178226863
:1063CC00890052181068C6490840C649014311603B
:1063DC00002B00D12BE72821794361180A005F328A
:1063EC00B5E7059A2A67049AB60096193268BE4931
:1063FC000A40802189015140BC4A0A433260D5E7EA
:10640C00049AB60096193168B54A1140B54A0A4348
:10641C003260187826688300F3181B685B040ED56D
:10642C00FFF796FD0190002800D100E72B005D33AB
:10643C00FF33FC351A88E96E03003000F5E6FFF7F0
:10644C009BFD0190002800D1F1E62B005F33EFE7B4
:10645C005531FF312068611800F078FD02E7012BFF
:10646C0000D036E7337DA249DB005B181A6892B284
:10647C001A60337DDB005B181A6829E7737D002BEB
:10648C0010D1337D9A49DB005B185A68920192094E
:10649C005A608022337D1206DB005B1859680A4370
:1064AC005A6016E7012B00D013E7337D9049DB00CF
:1064BC005B185A6892B25A60337DDB005B185A68DD
:1064CC00EEE780230398039A5B00357D18401A424F
:1064DC0019D1874AEB009B181B68F26A9B019B0D34
:1064EC009A4202D82900F062F7E6D21AF262B26A36
:1064FC001431D218B262326B6118D318336320682E
:10650C0000F024FDB0E52368029A039340231A405F
:10651C000192029A28001A4200D1EDE0FFF718FD13
:10652C008022F36AD201834214D80023F362029BC7
:10653C0013400193737D002B52D0012B5FD16C4A19
:10654C00ED00AD182B689BB22B60337DDB009B18E4
:10655C001A6853E01B1AF362029B134200D087E0C7
:10656C0028227A43A218150038352B78012B00D03D
:10657C0006E1936A1B189362336B1B183363516BE0
:10658C00536A99427ED3C91A516328227A43A218BE
:10659C00517D002900D092E0117D554EC90089191A
:1065AC0008688001800908603E2B75D91F201840AF
:1065BC00454268415909091A107D8A068021C0009C
:1065CC008019056809062A430A4302602821794389
:1065DC0061188A8B9BB2896A206800F083FCCFE03B
:1065EC00434AED00AD182B689B019B092B60337D52
:1065FC00DB009B188022196812060A431A602822B5
:10660C007A43A218517D137D002924D13848DB0030
:10661C001B185968890189095960137D8022DB0098
:10662C001B18596812060A435A6028257D436519C0
:10663C002000297D03F0D8F9019B002B00D19FE0AD
:10664C002A7D236892009B181968254A1140294A13
:10665C000A431A6094E00129E7D12548DB001B1896
:10666C00596889B25960137DDB001B185A68DBE747
:10667C00039BAD005D192A68194B1A401D4B13433F
:10668C002B606DE7002902D1030029707DE7002300
:10669C002B7053630B0078E7117D154AC9008918DC
:1066AC00002B05D180220868120602430A608DE790
:1066BC0001205A081840121892060868F5E70129BB
:1066CC0084D1117D0A4DC9004919086880B208604F
:1066DC00127D1904D200521910680143116075E73C
:1066EC008F8FFF07C08000008FBFFF0780800000E6
:1066FC000098004080C00000FFF73EFC8022F36A47
:10670C00D20183424CD2019BF362029B1340019352
:10671C0028237B43E3185A7D002A00D08DE0B14931
:10672C00ED006D182A68920192092A6080221B7D67
:10673C001206DB005B1819680A431A6028227A4398
:10674C00A218517D137D002900D084E0A548DB0000
:10675C001B185968890189095960137D8022DB0057
:10676C001B18596812060A435A6028257D4365197F
:10677C002000297D03F038F9019B002B00D15FE745
:10678C0028237B43E3181A7D236892009B181A6810
:10679C0095490A4030215140944A0A431A6063E4F7
:1067AC0002991B1A1140F3620191002BB0D0019B8E
:1067BC00002B08D1039BAD005D192A688C4B1A4045
:1067CC008C4B13432B6028227A43A21815003835C2
:1067DC002B78012BD4D1936A1B189362336B1B1843
:1067EC003363516B536A994242D3C91A51632822BD
:1067FC007A43A218517D002957D1117D794EC900D9
:10680C00891948688001800948603E2B3AD91F20BD
:10681C001840454268415909091A107D8A068021A1
:10682C00C0008019456809062A430A4342602821A2
:10683C0079436118CA8B9BB2CDE6012A00D07DE763
:10684C006849ED006D182A6892B22A601B7DDB0046
:10685C005B181A6871E7012987D16248DB001B18A5
:10686C00596889B25960137DDB001B185A687BE7A5
:10687C00002902D103002970B9E7002353632B7060
:10688C000B00B4E7117D574AC9008918002B05D1BC
:10689C0080224868120602434A60C8E701205A0861
:1068AC001840121892064868F5E70129BFD1117DEE
:1068BC004C4DC9004919486880B24860127D1904D2
:1068CC00D2005219506801435160B0E742050DD512
:1068DC0022684949536C20000B405364FDF752F970
:1068EC002900200003F071FCFFF7C4FB420406D51D
:1068FC0022684249536C0B405364FFF7BBFB802268
:10690C00010092011140104203D022683C49536CA3
:10691C00F1E7C20418D52068026C9A43026408207F
:10692C002268136C83431364B3239B00E25C012A3B
:10693C0003D12000E15403F06DFD2000FDF756F962
:10694C0022683049536CD6E7020512D5082221681B
:10695C00086C02430A6421682B484A6C02404A6462
:10696C0021680A6C13430B642000FDF731F9FFF723
:10697C0081FB020621D5216824484A6C02404A64F6
:10698C00B3229200A15C0029EED12168086C03436C
:10699C000B6408232168086C03430B640121A15488
:1069AC003C22236820005B6D9B081340B4229200AC
:1069BC00A35003F02FFDFFF75DFB830509D522687B
:1069CC001349536C20000B40536403F0FDFBFFF79D
:1069DC0051FBC00501D4FFF74DFB22680D49536CE8
:1069EC0089E7C04600980040BF8FFF0780800000F9
:1069FC008F8FFF0780C00000FFFB0000FFBF00006F
:106A0C00FFDF0000FFEF0000FFF700007FFF00003A
:106A1C00FFFD0000FFFE000003000020014A586447
:106A2C001A64704780BF0000036C024A1340036471
:106A3C00002070477F40FFFFF7B50D789F4AAD00EF
:106A4C0045192C6803001440CA780192032A04D813
:106A5C001000F9F737FB054846430122019202E08A
:106A6C00802292001443964A14432C600F78954D63
:106A7C00BE009E1934682C403C43144334600E7B9A
:106A8C000C78002E00D08DE08F4F4E78E400E41986
:106A9C00002E30D02668360C360426600E78CC8852
:106AAC00F600F6193768A408A4003C4334600C784F
:106ABC00A4001C192668760604D526682E40834D42
:106ACC00354325600C78C978A400814D1B19012928
:106ADC000BD020211C682C40614008E0C022D20061
:106AEC0014430022BAE78022F9E7196829400A43C7
:106AFC001A600198FEBD6668360C36046660724CEE
:106B0C000E782000F6003619CC887768A408A4000B
:106B1C003C4374600C78E40024186668B601B6092E
:106B2C0066600E690C783E2E24D91F20770906402A
:106B3C00300046424641BF1B634EE400A419BE061A
:106B4C00802760683F0606433E4366600C78A400CD
:106B5C001C192668760404D526682E405D4D3543F5
:106B6C00256009785C4D002916D1C0211C682C4089
:106B7C008901B1E75448E4002418002E03D1802683
:106B8C0067683606E0E7012077080640BF1966689B
:106B9C00BF0637436760D9E789005B181C68802102
:106BAC002C40E5E7CE78A4001C19022E55D127689D
:106BBC004A4E2F403E43444F266038000C78E40088
:106BCC00E4192668360C360426600E780C89F6001B
:106BDC00F6193768A408A4003C4334600C78E40030
:106BEC0024186668360C360466600E784C89F600FC
:106BFC0036187768A408A4003C43802774600C788E
:106C0C004878A400324EFF011C1900282AD12068B4
:106C1C00384206D027682F40BC4660462D4F0743AC
:106C2C0027600C78A4001C1927687F0604D52768F8
:106C3C002F40264D3D432560C0250C782648A400E6
:106C4C001C192768AD0107407D4015432560097864
:106C5C0089005B181968314049E72668204F3E408F
:106C6C001643A8E72068384206D027682F40BC4658
:106C7C006046184F074327600C78A4001C1927683E
:106C8C007F0604D527682F40104D3D4325600C78B6
:106C9C00CD78A4001C19012D0CD025682E40202580
:106CAC0075401543256009780B4889005B181968F5
:106CBC0001401CE725683540F3E7C0468F89FF0784
:106CCC00808000008F8FFF0700980040C08000007C
:106CDC00BF8FFF0780C000008FBFFF0780810000BF
:106CEC008F8EFF07F0B50B780C7B9B004D78414ADB
:106CFC00C318002C22D11C68002D11D0640605D5B8
:106D0C001D683D4C25403D4C2C431C600B789B0072
:106D1C00C31819683A4801400A431A600020F0BDB4
:106D2C00640405D51D68344C2540364C2C431C603E
:106D3C000B789B00C31819683348ECE780262E4C5F
:106D4C002F4FF601002D27D11D68354204D01E6847
:106D5C002C4D264035431D600B78284D9B00C318E5
:106D6C001E68760603D51E6826402E431E600B78DF
:106D7C009B00C3181E68344025431D600B78224DC0
:106D8C009B00C3181C682C4014431C600B789B00A0
:106D9C00C31819683940BFE71D68354204D01E6816
:106DAC00184D26402E431E600B789B00C3181E689E
:106DBC00760606D51E682640B44665460F4E2E4311
:106DCC001E600B780F4D9B00C3181E683440254382
:106DDC001D600B789B00C3181C683C4014431C605E
:106DEC000B7809499B00C01803680B401A430260DA
:106DFC0094E7C046808000008F8FFF07C0800000A2
:106E0C00BF8FFF0780C000008FBFFF070B780B4AB6
:106E1C009B00C0184B780168002B07D0084B194019
:106E2C0010234B401343036000207047054B19405F
:106E3C0080235B014B401A430260F5E78080000021
:106E4C00BF8FFF078FBFFF0710B50B7B002B1CD12B
:106E5C000B784A789B00C318002A18D01A6852067F
:106E6C0005D51C68154A1440154A22431A60CB7884
:106E7C00012B0AD00B7813499B00C3181A680A40DF
:106E8C0020215140104A0A431A60002010BD1A6894
:106E9C00520405D51C68094A14400C4A22431A6056
:106EAC000B780B4A9B00C01803681340C022920158
:106EBC005A40054B13430360E7E7C0468F8FFF072B
:106ECC00C0800000BF8FFF078080000080C00000E2
:106EDC008FBFFF07836D024A134083650020704704
:106EEC00FF7FFFFFF7B50324D81C23401C00651E51
:106EFC00AC418008001B144C0D00121904000192C7
:106F0C00002C0FD1002B0CD02500800009184E5DF1
:106F1C00EF00BE4001353443AEB2B342F7D1121884
:106F2C001460F7BD2E78013CB44667466E78360285
:106F3C003E43AF783F043743EE78043536063E4384
:106F4C00019F40C70197DBE700980040F7B50C00A4
:106F5C0049780600227B012900D09BE12069A569B4
:106F6C00854200D90500002A20D1ABB2E2886169C4
:106F7C003000FFF7B7FF2378C049DB005B181A68B5
:106F8C002D0492B21A602378DB005B181A68154343
:106F9C001D602378BA4A9B00F318196811403022FF
:106FAC004A40B8490A431A600020FEBD2278E778AF
:106FBC009100236A7118022F00D040E10A689842B0
:106FCC0000D336E1B04B40201A40B04B13430B605A
:106FDC00236A22785B1B23629300F3181B68617889
:106FEC009C461F00ABB2019363460740034200D19D
:106FFC008DE000295AD1A149D20052180B005168DA
:10700C0089018909516021783E2D3FD921382840CA
:10701C0047427841C9006A09C918121A4868920691
:10702C0002438020000602434A6062896169ABB268
:10703C003000FFF757FF636921695B196361236AAD
:10704C0000228B4201D95A1B2B0022626278002A43
:10705C004CD12278894FD200D21911688901890943
:10706C00116021783E2B31D91F20184045426841D0
:10707C00C9005A09C919121A0868920602438020DD
:10708C00000602430A609BB222898CE07B4BC9004C
:10709C00C918002D03D1802248681206C3E70120CD
:1070AC006A082840121892064868BCE70129BCD12E
:1070BC007248D2001218516889B2516022782904A2
:1070CC00D2001218506801435160AEE76B4AC900F8
:1070DC008918002B03D1802208681206D1E7012001
:1070EC005A081840121892060868CAE7012ACAD131
:1070FC0022786248D2001218116889B21160227885
:10710C001904D2001218106801431160BBE7002962
:10711C005ED15A49D200521811688901890911604F
:10712C0021783E2D44D91F20284003005842584155
:10713C006A09121A5148C9000918086892060243D4
:10714C008020000602430A602289ABB230006169DC
:10715C00FFF7C8FE636922695B196361236A934276
:10716C0001D95F1B2B0062782762002A50D122784C
:10717C00424FD200D2195168890189095160217896
:10718C003E2B35D91F20184045426841C9005A0989
:10719C00C919121A4868920602438020000602435D
:1071AC004A609BB2628930006169FFF79BFEF0E692
:1071BC00324BC900C918002D03D180220868120671
:1071CC00C0E701206A082840121892060868B9E73F
:1071DC000129B9D12948D2001218116889B211605D
:1071EC0022782904D2001218106801431160ABE711
:1071FC00224AC9008918002B03D180224868120644
:10720C00CDE701205A081840121892064868C6E7C4
:10721C00012AC6D122781948D2001218516889B2B5
:10722C00516022781904D200121850680143516041
:10723C00B7E717480240134802430A6058E75B1B44
:10724C0023620868ABB229040C4DD20052194006D7
:10725C0009D5506880B250602278D200521950681B
:10726C00014351609EE7106880B210602278034899
:10727C00D200121810680143116005E70098004015
:10728C00BF8FFF07808000008F8FFF078081000079
:10729C008F8EFF07002A22D1A36921698B4201D965
:1072AC005A1A0B00A2612278844DD20052195168EF
:1072BC0089018909516022783E2B00D8ECE01F200F
:1072CC005909034058424341C91A8B068021D20008
:1072DC0052195068090603430B43536075E0E37879
:1072EC00022B00D08DE000291AD12378734DDB00DE
:1072FC005B191A68920192091A60226923783E2A56
:10730C002DD91F205109024050424241891A8A0648
:10731C008021DB005B191868090602430A431A60D6
:10732C0062782378002A5DD1644DDB005B195A68C2
:10733C00920192095A60226923783E2A21D91F2092
:10734C005109024050424241891A8A068021DB00D1
:10735C005B195868090602430A435A6022E05749F0
:10736C00DB005B18002A03D1802219681206D5E7CE
:10737C0001205108024089181A68890611431960C6
:10738C00CEE74E49DB005B18002A03D180225968F6
:10739C001206E1E701205108024089185A68890653
:1073AC0011435960E3692278002B0ED09200B21879
:1073BC00136843490B408B4201D0002B05D1116857
:1073CC00404B1940404B0B43136023783F4A9B00C2
:1073DC00F61833681340C02292015A403C4B1343B9
:1073EC003360E1E5012ADDD13449DB005B185A68D2
:1073FC0092B25A6023782269DB005B185968120438
:10740C00AAE70120834200D0CFE5A36922690020BE
:10741C00934201D9981A1300A061002919D122783E
:10742C00264FD200D219116889018909116021787F
:10743C003E2B21D91F20184045426841C9005A09EA
:10744C00C919121A086892060243802000060243EA
:10745C000A6061782278002900D125E70129B4D18E
:10746C001648D200121851681B0489B25160227858
:10747C00D200121851682FE7104AC9008918002B46
:10748C0003D1802208681206E1E701205A0818404F
:10749C00121892060868DAE70849D2005218002B35
:1074AC0003D1802351681B0616E7012059080340BD
:1074BC00C918536889061943516086E70098004043
:1074CC00404000008F8FFF07C08000008FBFFF0778
:1074DC0080800000F7B50324D81C2340134C80088F
:1074EC0012191C00651EAC41001B0D00040001921A
:1074FC00002C0ED1002B0BD080001218091810682C
:10750C000500E200D5400D550134A2B29342F7D1EB
:10751C00F7BD019F013C40CF0197370A2E706F7069
:10752C00370C360EAF70EE700435E1E70098004072
:10753C000F4B411E02000120994217D80D4902231E
:10754C008A4203D80C4B93429B415B4207200B4968
:10755C000A6882431A430A600A680240934201D0C7
:10756C000A680240981A421E9041C0B27047C04649
:10757C00FF8FD003006CDC0200366E01002002404D
:10758C0010B50400FAF732F803480121034A02F05F
:10759C00B8F8200002F089FFB0AD000846C600081C
:1075AC00F0B585B005000C0000AFEFF310837B60E5
:1075BC0072B62D4A9368FB602C4B042802D82C4BD6
:1075CC008100CB586E468AB0117C6A46D361294B38
:1075DC0029489384294B5061956111621361B12143
:1075EC00274B1032BB60B86800238901FAF704F905
:1075FC00B546002C07D0E369DB0504D00121214AF4
:10760C00B86802F07EF8FB68002B07D0180002F077
:10761C00B8FF002802D00378002B00D11A486E4620
:10762C008AB06A46194BD0615361FB689361114B68
:10763C001384174B136191210023114810328901D7
:10764C00FAF7DAF82100B5462800FFF799FF7B68B6
:10765C00002B02D162B6BFF36F8FF868FBF77AFC90
:10766C00BD4605B0F0BDC046E013002055C600086D
:10767C0004B10008010300006BC6000805000001FE
:10768C00B0AD000893C6000863C60008B4C6000875
:10769C0004000001F8B501270A4E83009D59013002
:1076AC0084003359AB4200D8F8BD6868002806D076
:1076BC00037F3B4201D102F0D2FE0835F1E72B6883
:1076CC009847FAE718B10008012270B5234B032044
:1076DC0086B01A70FFF7DEFF01F0B6F90420FFF751
:1076EC00D9FF1F4C26001F4DAC420ED300F05CFDA1
:1076FC00AE4220D300F068FDF8F78AFE01211A4A49
:10770C00137B8B43137306B070BD636A0593236AB6
:10771C000493E3690393A369029363690193236957
:10772C000093E368A2686168206800F02FFB23686F
:10773C005C653034D7E7B26AF36A511C01D1591C2D
:10774C0005D011003068194303D100F013FE303618
:10775C00CEE70649183000F0A9FFF8E76C140020BA
:10776C0088AC000888AC00088006002077A60008CA
:10777C0070B5702601250400464301021148802291
:10778C000918002086B004950E3503950535654320
:10779C000D4B0590029001900C48F6182D180C4BCF
:1077AC0030000095520000F0F1FA0422737B2C7427
:1077BC00934373730134074BE402E418EE606C607E
:1077CC0006B070BD701F002010060020E0130020D2
:1077DC00BFA4000870170020F0B5002087B0FFF799
:1077EC0059FF214B83F308882049214B0A6A002555
:1077FC001A40C0231B0413430B62FBF77FFBFBF700
:10780C0097FCF9F757FE1B4800F026FBF9F710FD23
:10781C000120FFF73FFF0220FFF73CFF00F004FDC3
:10782C00154C164B80225C61154B164E05930123AB
:10783C0015490493520133002000039502950195DC
:10784C00009500F0A3FA04220700637B2000934309
:10785C00637302F0D4FE2800FFF78AFF3200390070
:10786C002000FBF749FCC046701F002000ED00E033
:10787C00FFFF00FF8007002080060020E01300209F
:10788C00D8B50008D576000870200020F0B585B07A
:10789C0004001F000392EFF3108672B6C368354ADA
:1078AC00002B0ED080689168884217D0039B3B4315
:1078BC001AD1002E02D162B6BFF36F8F1020404256
:1078CC000AE09168897B49B20133E36093682161D6
:1078DC00A360002E04D0002005B0F0BD2169F3E7B1
:1078EC0062B6BFF36F8FF6E70E23897BC35649B29E
:1078FC00994200DD19000A007F3201DA7F214942EA
:10790C0000258B4202DD02F0DBFD05001A4B220044
:10791C000293039B310002980093019700F088FBBF
:10792C000028D8D0EFF3108672B6A068002819D0C2
:10793C00236821699C420BD0002B09D09B7B5BB246
:10794C00994200DD19000B007F3301DA7F21494297
:10795C0002F0B6FD002805D03100029800F0F8FBCB
:10796C000B20ACE7002DF7D1002EF9D162B6BFF396
:10797C006F8FF5E7E01300206D140020F8B58368D5
:10798C000500002B3CD0214A926893423BD1C3683E
:10799C00012B03D9013BC3600020F8BDEFF3108726
:1079AC0072B60169806802F08BFD2C68AC4208D17C
:1079BC000023AB60EB609F42EED162B6BFF36F8FDA
:1079CC00EAE7002CF4D062682368002613605A6042
:1079DC0002222000637B2660934363736660A6607B
:1079EC00183002F08CFE0E23AC60E35620002B61A5
:1079FC00E66602F004FE3900054800F0A9FBCBE76F
:107A0C0016204042C9E70120FBE7C046E0130020E6
:107A1C006D14002070B5EFF3108572B60468A042A7
:107A2C001AD0002C18D062682368002613605A60A4
:107A3C0002222000637B2660934363736660A6601A
:107A4C00183002F05CFE2000E66602F0D8FD29003A
:107A5C00084800F07DFB70BD8268C3689B1A591EF4
:107A6C008B419B188360002DF5D162B6BFF36F8FED
:107A7C00F1E7C0466D14002013B50400EFF310813C
:107A8C0072B68068002808D00138A060002902D1A5
:107A9C0062B6BFF36F8F002016BD1000184307D1DC
:107AAC00002902D162B6BFF36F8F10204042F3E77A
:107ABC00009201932200024800F0BAFAECE7C046AB
:107ACC006D1400200123802213B5054C054906488E
:107ADC0000945B42D20000F015F9002016BDC046A0
:107AEC0030B1000870300020F0060020F0B5050021
:107AFC0087B0EFF3108772B62E006C6F8C36002CAB
:107B0C001CD10221300002F0FAFC002866D02C00B7
:107B1C00843400220121200002F0D3FD0028F8D18A
:107B2C000023029301225242D317009201932A00A0
:107B3C0039007C323C4800F0D9FCDAE72368AA6FA4
:107B4C006B67944200D1AB670222336813433360F6
:107B5C000423E2689A43033B1343E3606368002FFA
:107B6C0047D020009847EFF31083059372B6E36873
:107B7C0001211A008A43100908423ED1E260E368F1
:107B8C009A071AD502229343E360284B1868002801
:107B9C0013D00021026800280FD04768BC423AD1AC
:107BAC000268002931D159681A60814200D15A60AB
:107BBC00002303600830FFF72DFF02223368934344
:107BCC00059A3360DB05DB0F002A02D162B6BFF3E6
:107BDC006F8F002B8DD100F031FB8AE73368DB0609
:107BEC009ED53060002F02D162B6BFF36F8F07B005
:107BFC00F0BD62B6BFF36F8FB3E711229343E3601E
:107C0C0020001030FFF706FFB9E70A605A6882427D
:107C1C00CED15960CCE79446002A01D011688C462D
:107C2C00010010006246B6E76D140020001400201D
:107C3C00F7B5C3680D00590801220F000400174066
:107C4C0011424CD19B0813421ED12B68002B01D141
:107C5C0083682B600127E3683B4202D0A368FF19BD
:107C6C002B602E68002E48D03100254B8C319A6841
:107C7C00336F01919A4222D00A68012193080B407C
:107C8C000A4204D113277F4200232B6015E0002BFE
:107C9C0025D1D3080B40002B21D100232360B36FD7
:107CAC00002B27D1B4677467300002F034FC042336
:107CBC00E2681343E3602B68A3603800FEBD02F05A
:107CCC0057FC019B01221B6800280AD1D9081140DE
:107CDC001342D7D00029E0D09B081342DDD11027E6
:107CEC00D1E7990811401342CCD00029F7D1DB0819
:107CFC001340D0E71C60B467D6E71627C3E7C0462D
:107D0C00E0130020F0B5040000206067A06720009D
:107D1C0089B07C30261D0E9DE067F067083000604E
:107D2C0040600120002D07D0287946427041FF2683
:107D3C004042B0430230FF3026008C3630600126C2
:107D4C007642F7170696079700260F48039304967A
:107D5C000300029620000196009400F051F8B54201
:107D6C000CD02968B14202D0200002F007FC6B79DC
:107D7C00002B03D00123227B13432373200000F03C
:107D8C00F9FA246709B0F0BDF97A0008F0B587B0AC
:107D9C000593030058338365C365109B0727037352
:107DAC00042300250732BA434373D2190F9BBA43FD
:107DBC0083738B180E0085601900C5738561C561CE
:107DCC0004000493FAF7D2FF049BC019B8431F1A9E
:107DDC000E9B3A0002930D9B310001930C9B2000EB
:107DEC000093059BFBF772F9044B65659B68AB42EE
:107DFC0000D01B6E3800236607B0F0BDE0130020E6
:107E0C0070B50400002086B005900E98119D04906A
:107E1C000D98109E03900C9802900B9801900A9864
:107E2C0000902000FFF7B2FF2B00721C01D1013330
:107E3C0005D02B00334305D1200000F09BFA200025
:107E4C0006B070BD200032002B000249183000F043
:107E5C002DFCF4E777A60008022310B50400FF33CD
:107E6C00838100F0EBFD014B9C6010BDE013002002
:107E7C000B21084A49429368D966986680230649C3
:107E8C005B05486803434B6062B6BFF36F8F936822
:107E9C00D86E7047E013002000ED00E00D2370B5A4
:107EAC00C356427B002B38DBD30636D180235B4292
:107EBC0013431B4C4373A3691A49E2698B4207D1E4
:107ECC00016042601060E06111E09A42F8D01B68DA
:107EDC00002BF5D00E250E2645579E57B542F4D0F3
:107EEC00AE42F2DD5A680360426010605860A569CA
:107EFC008D4201D0002D00D1E568A3685A7BD206D3
:107F0C0005D1DA897F2A02D9AA69002A06D0AB42A8
:107F1C0002D0280000F02CFB656170BD6361FCE7AA
:107F2C00E0130020F81300200D2270B582560500D6
:107F3C00437B002A04DA7F221340437302F023FBB5
:107F4C000D4E0E4AB469B368944201D0002C00D196
:107F5C00F468AB4208D05A7BD20605D1DA897F2A65
:107F6C0002D9A269002A05D0A34202D0200000F059
:107F7C00FFFA2300736170BDE0130020F81300209A
:107F8C0010B5511C01D1591C03D00249183000F016
:107F9C008DFB10BD77A600080D2270B5825604002B
:107FAC00437B002A04DA7F221340437302F0EBFA7E
:107FBC008023627B5B4213431B4D6373AB691B498C
:107FCC00EA698B4207D1216062601460EC6111E0B8
:107FDC009A42F8D01B68002BF5D00E200E262056A6
:107FEC009E57B042F4D08642F2DD5A68236062603C
:107FFC0014605C60AE69AB688E4201D0002E00D17B
:10800C00EE68A34208D05A7BD20605D1DA897F2AC2
:10801C0002D9B269002A05D0B34202D0300000F078
:10802C00A7FA33006B6170BDE0130020F813002039
:10803C0070B50C0011000A4A0A4B90681860EFF3F7
:10804C00108372B69568280002F0B0FA049A059B6A
:10805C002800FFF795FF2000FFF70AFF70BDC04610
:10806C00E013002008140020F7B50400EFF310878C
:10807C0072B61F22437B1A4050425041C0B201904D
:10808C004DB2002A3CD17F3213406373200002F0C2
:10809C007AFA8023627B5B4213432B4EA573637386
:1080AC00B3692A498B4229D1F2692160626014605C
:1080BC00F4610FE09A42F8D01B68002BF5D00E202B
:1080CC0018568542F6D0A842F4DD5A6823606260E7
:1080DC0014605C60B4698C4201D0002C00D1F4684F
:1080EC00B3689C4202D0200000F042FA7461002F69
:1080FC0002D162B6BFF36F8F0198FEBDF269DCE767
:10810C009B071FD5A668200002F03DFAA5733368C3
:10811C009E4209D17368266063601C607460E6E758
:10812C0072689342F6D01B68002BF3D00E229A563D
:10813C009542F5D0AA42F3DD5A6823606260146060
:10814C005C60D4E7A573D2E7E0130020F81300209D
:10815C0010B500290AD1EFF30580002807D1064B92
:10816C009A685B699A4202D0FFF782FE10BD62B634
:10817C00BFF36F8FFAE7C046E013002010B500285C
:10818C000AD1EFF30580002807D1064B5A699B688A
:10819C009A4202D0FFF76CFE10BD62B6BFF36F8F30
:1081AC00FAE7C046E0130020EFF3108172B6054BDE
:1081BC009A68D37B013BD373002902D162B6BFF31B
:1081CC006F8F7047E013002070B5EFF3108672B616
:1081DC00134DAB68DA7B0132DA73AC69114A944205
:1081EC0001D0002C00D1EC685A7BD20605D1DA897B
:1081FC007F2A02D9A269002A05D0A34202D020000E
:10820C0000F0B6F923006B61002E02D162B6BFF309
:10821C006F8FEFF3108072B6FFF7B0FF70BDC046E2
:10822C00E0130020F8130020024B034A9A61DA6134
:10823C007047C046E0130020F813002070B5EFF330
:10824C00108572B61C4CA168E3690A68CB1A581EDB
:10825C00834149685B420A6051601340E169A2683E
:10826C00002B05D1154B516013600A60E2610CE0E4
:10827C000E200E2610569E57B04218D0864216DDA0
:10828C005968136051600A605A60A6690B4B9E4294
:10829C0001D0002E00D1E668A3689E4202D03000C7
:1082AC0000F066F928006661FFF7E2FD70BD8B42B5
:1082BC00D8D01B68D4E7C046E0130020F813002088
:1082CC00F8B5030007000C000B4303D1FFF7B6FF12
:1082DC000020F8BDEFF3108672B6134D134BA8684F
:1082EC001860FFF721FEA86823003A0010491830E7
:1082FC0000F0DCF90423AA680400517B30000B4326
:10830C005373FFF7B5FDAB689A6A002AE0D180225F
:10831C00DB6A12069342DBD102F017FA201AC34330
:10832C00DB171840D5E7C046E013002008140020E6
:10833C0077A6000870B504000D00FFF7C1FF01001F
:10834C002000631C01D1013510D00A00CB17092085
:10835C000021801859410A220023F7F797FF0029C2
:10836C0003D180231B06984200D3014870BDC04640
:10837C00FFFFFF7F70B50400EFF3108572B6042683
:10838C00437B33420DD0183002F0B9F9637B2000E7
:10839C00B3436373FFF782FD29000548FFF7D8FE4E
:1083AC0070BD002DFCD162B6BFF36F8FF8E7C046ED
:1083BC006D140020014B98687047C046E0130020F4
:1083CC00F0B5037B85B004000393EFF310830193A6
:1083DC0072B6019B02930823427B1A4207D0019B81
:1083EC00002B02D162B6BFF36F8F05B0F0BD190040
:1083FC00114348B2002857DB6173A368002B02D0ED
:10840C00200002F0C8F820002600183002F077F99E
:10841C005836A56DAE4201D0002D4DD1304F002500
:10842C00BB689C4204D1EFF305856A1E9541EDB201
:10843C00BE692C4A964201D0002E00D1FE68B34290
:10844C0002D0300000F094F820007E6101F056FA62
:10845C00002D02D02448FFF7FFFCBB689C4238D1AA
:10846C00EFF30583002B34D1237BDB070FD5019B66
:10847C00002B02D162B6BFF36F8F62B6BFF36F8F62
:10848C000423181C02DFEFF3108372B602930298D8
:10849C00FFF7EEFC039BDB07A7D562B6BFF36F8F2C
:1084AC000423181C02DFA0E77F210A40134320009D
:1084BC00637302F068F8A0E7280002F06CF828005B
:1084CC00183002F01CF900232800EB66FFF7E6FCDD
:1084DC009FE7019B002BDDD162B6BFF36F8FD9E70D
:1084EC00E0130020F81300208007002073B5069DD0
:1084FC00079E089C00950196FFF79AFD002C03D06F
:10850C00024B9B681B69236076BDC046E0130020BC
:10851C000121044B044AC01A044BC0104343D154EC
:10852C007047C046F00700206D140020ABAAAAAA21
:10853C00C289030000207F2A11D80A4A106800283B
:10854C000DD00E21084A595612680020914206DBC4
:10855C005A7BD20603D10548181A431E98410123B1
:10856C0018407047340000200C1400201006002026
:10857C0070B518240C4B05001E7C0C4B7443E4188E
:10858C00200002F0BCF80022094B28009A55FFF796
:10859C00CFFF002807D0074B20001A680649013A84
:1085AC00D31700F083F870BDE0130020F007002013
:1085BC006D140020340000201D85000870B5EFF309
:1085CC00108572B6104A114B94681868A04207D1F6
:1085DC00FFF7CEFF002D02D162B6BFF36F8F70BDD7
:1085EC0000211960127C0A4B9B5C8B42F2D020005C
:1085FC00FFF79EFF0028EDD0637BDB0602D1200045
:10860C00FFF7CAFC2000E3E7E01300200814002069
:10861C006D140020024B1868984200D1002070475E
:10862C003800002070B50600FFF7F4FF002810D0CA
:10863C00026943693400F517121BAB41002B08DCAF
:10864C0003D1802109068A4203D2D843C0171040B7
:10865C0070BD0148FCE7C046FFFFFF7F002010B54E
:10866C00034B1B68834201D1FDF702FC10BDC046D1
:10867C001014002030B500280ED00B4B5B689842CC
:10868C000AD00168002907D00A694B690469456959
:10869C0012196B410A614B610368426813605A609E
:1086AC0000230360436030BD38000020F0B50400A7
:1086BC0015001E0085B0531C02D1731C00D17CE048
:1086CC00A160EFF31083039372B6002E26DBFFF745
:1086DC00C5FF00210090012040197141009AD31769
:1086EC0012184B41364922616361086849681218B7
:1086FC004B411E00150001230293FFF78BFF07006F
:10870C00304B9C465B680193002F1DD16346236060
:10871C00019B63601C6063465C6027E0284B186813
:10872C00596802225242D317121A8B41521BB34181
:10873C001100002B04DC01D1002A01D101210023FE
:10874C00636121610023D7E738697969226963691C
:10875C00994202DC28D1904226D9801A99417B6833
:10876C0038617961636027601C607C60FFF752FFA1
:10877C0084420FD1144B1B68002B0BD1029B002B96
:10878C0002D1FFF76BFF00900098FFF74BFF002121
:10879C00FDF7E4FA039B002B02D162B6BFF36F8F97
:1087AC002800310005B0F0BD121A8B4122616361C3
:1087BC00019B9F42AAD03F68A6E700250026EFE761
:1087CC00080800203800002010140020F0B587B0F5
:1087DC00EFF3108372B601932F4B1860FFF71AFF5B
:1087EC002E4F04003A687B68029203932A4B9C46F6
:1087FC001D6800280FD042690669EB179A4202DC0B
:10880C0024D1AE4222D91900226963692800121AB8
:10881C008B4122616361029803992A00EB171218AD
:10882C004B4100243A607B60634620001C60FFF7DC
:10883C00F9FE2100FDF792FA019BA34202D162B628
:10884C00BFF36F8FFFF7BAFE07B0F0BDF3170496B6
:10885C000593049A059B02980399801859410023AB
:10886C0000220E4D22616361286069602000FFF7D1
:10887C0001FF019B002B02D162B6BFF36F8F20006A
:10888C00A3689847EFF3108372B6034A01931368F9
:10889C009B1B1360A2E7C0461014002008080020A0
:1088AC0010B5EFF3108472B6FFF7D8FE020006493C
:1088BC00C3170868496880185941002C02D162B668
:1088CC00BFF36F8F10BDC04608080020F7B5040039
:1088DC00EFF3108572B603680195002B05D0002DBF
:1088EC005CD162B6BFF36F8F58E00122C16A806A17
:1088FC00002312184B41002B01D1012A33D9012638
:10890C007642F71736184F41002F01DA0026002760
:10891C0001F01FFF01220023801859418019794171
:10892C00002902DC3BD1002839D001F012FF0023D2
:10893C0001228018594180197941244B994201D167
:10894C00033030D801F005FF012200238018594173
:10895C0002225242D31780197941121A8B412000FE
:10896C001B49FFF7A3FE236B01332363236A002B00
:10897C000BD0002D02D162B6BFF36F8F2000236A9B
:10898C009847EFF3108372B60193A5691834A5428A
:10899C0001D0002D0BD1019B002BA2D0F7BD0222E0
:1089AC005242D317DBE7802300221B06D7E72800AF
:1089BC0001F031FE0023EB66019B002B02D162B665
:1089CC00BFF36F8F280001F01AFEE7E7FFFFFF7F70
:1089DC00D9880008F8B5060014001D00EFF31087C5
:1089EC0072B6511C07D1591C05D1002F02D162B6A9
:1089FC00BFF36F8FF8BD002B0DDB14001D1E05DCC3
:108A0C00002B01D1002A01D1012400250122524260
:108A1C00D317A4185D41300001F071FE069A079B34
:108A2C00B262F36200232200336330002B00024950
:108A3C00FFF73CFED9E7C046D9880008014B036616
:108A4C007047C046A400002010B5024800F081FB1E
:108A5C0010BDC04622C7000810B5064C064B9C4200
:108A6C0001D3002010BD2000A268616801F0C0FE97
:108A7C001434F3E7A4000020B80000200CB470B547
:108A8C008AB002AC05000E0020220021200001F06B
:108A9C00C0FE0223A3700D4B25616360002E13DB17
:108AAC0001D0731EED180FAA20000E99656101927A
:108ABC0000F00EF8002E02D0002223691A700AB0C2
:108ACC0070BC08BC02B018470025ECE775A900087B
:108ADC00F0B5436893B003900893837815009B0717
:108AEC0000D4F8E0002301930E78002E6AD0252ED6
:108AFC000DD04B1C0993019B013301930399089BE7
:108B0C00F0B29847002800DADFE00999ECE74E78DC
:108B1C008B1C0993252EEED0002304211C00099AEE
:108B2C000293079309921F2C2ED83000203810285E
:108B3C000AD8F7F7C7FA1D0909270909091E0909F7
:108B4C00091B0925090918003300303B092B29D9C9
:108B5C002A2E32D108CD600622D4002B29DB20200E
:108B6C000793044305E001231C4302E002231C434A
:108B7C000C43099B01321E78002ED3D109922DE0B3
:108B8C000823F1E71023EFE77F2C1ED83300303B8E
:108B9C00092BDDD8600605D50A20029E7043C31848
:108BAC000293E6E70A20079E7043C318079320231D
:108BBC00DAE75B4207932823D6E72E2E05D1402314
:108BCC001C42D1D0019813B0F0BD6C2E2DD027D8FB
:108BDC00682E31D06A2E32D04C2E30D0029B002B16
:108BEC0003DA40239C4300230293202333431A00CF
:108BFC00653A022A01D9612B24D10722EB1D93433C
:108C0C0008331D00AB4F0292240753D5019A029BE7
:108C1C0016009C18B4424FD1079B029A9E1A82E10F
:108C2C00742EA6D07A2EA4D0D8E780231C429BD0D9
:108C3C0080208000044397E780235B00F6E7A023A5
:108C4C009B0091E730006338122800D9E3E0F7F776
:108C5C0039FA0A46E2E2E2E246E2E2E2E2E2F3DD7D
:108C6C00E2E211E2AD0004CD0CAB1A7001230CAFA3
:108C7C000293C9E780CD002F00D18F4F0299630674
:108C8C0001D401214942380001F0DCFD0290BBE720
:108C9C0020200399089B9847002816DB013C029B77
:108CAC00A342F5D3079A019B944663441B1B019383
:108CBC000794ABE7079CF2E7019B0399FB1A985DBD
:108CCC00089B984701360028A4DA039B9A78042362
:108CDC001343039A937001235B42019372E72306BB
:108CEC003FD5A30537D50722073595432F000CCF69
:108CFC0004920593102325009D43059B002B3ADA23
:108D0C000499059A00244B429441049305948023C2
:108D1C00DB001D43ADB20CAC0A230498059922006C
:108D2C0001F09BFD041B6B0665D501232A009A43B9
:108D3C001300029AA24200DCA4E0002E00D19CE0B9
:108D4C001022290011400B91154200D09CE0029A90
:108D5C001D0006921EE02F0008CF0493DB1705932D
:108D6C00C8E72F0008CFE205F7D5A20501D55BB205
:108D7C00F3E71BB2F1E7049B059A1343CBD16306CF
:108D8C00C9D5029B002BC6D111339C43029B2500F5
:108D9C001C0006932A00494B1A400B921D4277D0B7
:108DAC00069B0133069300230B9371E010239C4325
:108DBC00063B9C46802322001A4006921C4242D05D
:108DCC0021008133FF3319401C4239D00722EB1D9F
:108DDC0093431F0003CB083703000B4346D12500F8
:108DEC0016339D43630644D5029B002B41D11733A8
:108DFC009C432500029C10232A001A400B921D4212
:108E0C0056D0631C002E42D022003FE0102378265F
:108E1C009C461C43CEE7782B04D110229B1B1A4393
:108E2C009446C7E725200399089B9847002800DA49
:108E3C004BE7019B023360E6082300269C46B9E70A
:108E4C002F0001CFC8E72F008022210008CF52004D
:108E5C00180011401442BFD0802221009200114012
:108E6C0098B21442B8D00699D8B2B5E706239C4301
:108E7C0025000CAC6346220052E711239D43029B54
:108E8C00069387E71D00B6E71D00029A931C069314
:108E9C002B072AD4EB0709D5079B069A0294934219
:108EAC0004DD9B1A1B190293079B0693069B10E08B
:108EBC0006946FE751C700084AC700080604000073
:108ECC0020200399089B9847002800DAFDE60A9BAE
:108EDC0001330A930A9A079B9342F1DC069A019B91
:108EEC009B1A0A9A9B18019306920B9B002B25D078
:108EFC0030200399089B9847002800DAE5E6019B8F
:108F0C00002E12D101330193019E029B019A9B18F2
:108F1C009B1BA34220DC2500002D25D13D00079B87
:108F2C00069AA4199E1A019431E002330193F0B20F
:108F3C000399089B98470028E6DAC6E6174B1D42B2
:108F4C00E2D02020AB0700D50B306D0500D52D20CD
:108F5C00019B01330193EBE730200399089B013609
:108F6C0098470028D1DAB0E60CAB013DE85C0399D8
:108F7C00089B98470028CFDAA7E6019B20200133F5
:108F8C0001930399089B9847002800DA9DE6019A03
:108F9C00A3199B1A002BF0DCB7E5C04606040000B1
:108FAC007047020010B50B001179012214008C409F
:108FBC0021000068046924680C4200D05340002B47
:108FCC0003D08368DB68984710BD83681B69FAE798
:108FDC00C9004018408840087047F8B50D000400DF
:108FEC00FFF7F6FFF7F714F91F21091A8A00A218E8
:108FFC00EB0010691F1D0633E719E318AEB2002809
:10900C0008D101308840E1680143E16015613E8080
:10901C001E80F8BDC1000431625A3A80D200A218F9
:10902C001880D6806652F4E70723F7B50027043A78
:10903C00CC1D89189C4399430B1BDE080460A66069
:10904C00E7603000009301912425F7F7E1F8202226
:10905C002D1A121A200039009200103001F0D9FBA1
:10906C000123AD000735ED086A001A436280711BBD
:10907C00EA00A0184B0027804380009BA552E21801
:10908C00019B578019800123F600A61972882900CC
:10909C00134373802000FFF7A0FFF7BDF0B585B038
:1090AC000D001C1E0290039229D000265B780193C0
:1090BC00E078237840009B00C018A378C0182018D3
:1090CC00019B9E4210D36279237912021A43A37931
:1090DC0003991B041343E279029812061A432300E6
:1090EC000833A84705B0F0BD0378471C9B00380037
:1090FC001F51F7F717F9013038180136E0E7162041
:10910C004042EFE770B500240200012520001378DF
:10911C00002B01D118000AE0002813D08C4207D193
:10912C00702B04D01E00403E3A2E0BD8002070BD90
:10913C001E00403E3A2E05D8537801320134002BE4
:10914C00E8D00020252B00D168400132DFE7002059
:10915C0070470FB407B504A901C9019100F080FA5A
:10916C0003B008BC04B0184770B5056908242E007C
:10917C000023020026401800254205D1D068136850
:10918C00984203D9C31A30000B6070BD126A0120DB
:10919C00D31AF9E713B501A90400FFF7E5FF00287E
:1091AC0004D0019BE268013B9B180193206A019B50
:1091BC00C01A013816BD10B5040050182269236A74
:1091CC00D20702D5013B184010BD9842FCD3C01AFF
:1091DC00FAE710B504000A00C168FFF7ECFF08229B
:1091EC002369E0609343236110BD022270B50D002A
:1091FC008B001A430368C1699B005A500400016834
:10920C002A00FFF7D8FFE3682060984203D10823B7
:10921C002269134323612A0061682000FFF7CBFF0A
:10922C00606070BDF0B51F00C3681600C2699B007A
:10923C00D518D25C032385B01A4004000023029198
:10924C00022A08D033603B600222236913420DD1FD
:10925C000023019339E02968336089083B60F3D01F
:10926C00FFF7B7FFE368A3600123F2E7A3692800C7
:10927C0098472B780090DA07D10F0191002AE7D09C
:10928C0002221A4003920222134221D0029B002B8D
:10929C0003D019002000FFF7A8FF61682000009A96
:1092AC00FFF789FFA368E1686060994206D120004E
:1092BC00009AFFF780FF0023A0600193A368226946
:1092CC002360E360082313432361019805B0F0BDCC
:1092DC0020000099FFF77DFFE368A360029B002B41
:1092EC0004D02368E26903999B009950029B009A71
:1092FC009C4662443A6021682000FFF75CFF08231B
:10930C00226920601343012223612B7893432B7035
:10931C003560A9E770B504000D001600FFF74BFF90
:10932C002368834205D10822236925609343236176
:10933C0070BD0223B2001343E269AD00AB5061680B
:10934C0032002000FFF737FF6060F1E770B503696A
:10935C0004005B0706D5456AFFF71CFF854200D267
:10936C000500656270BD70B50D0004001C22002163
:10937C0001F04FFA0022EB68A361AB6863612B68C4
:10938C00E3616B68626223622A69002B04D0591E68
:10939C000B4201D101231A4322612000012200213A
:1093AC00283001F09FF870BDF0B58BB00593002309
:1093BC000492026A04001E000291079309938A42E8
:1093CC003BD30193EFF3108772B6099A0397002AE7
:1093DC0005D020000199FFF79DFF00230993200081
:1093EC0008A9FFF7C1FE089B029A0500009393425F
:1093FC002BD32368E2699B00D618D35C03229343DA
:10940C00337021682000029AFFF7D5FEE3682060D4
:10941C00984215D00025039B002B02D162B6BFF3F6
:10942C006F8F0799002906D06369002B01D02000AB
:10943C00984700230793002DC4D130000BB0F0BD2A
:10944C000822236913432361E4E7002804D0200099
:10945C000099FFF7CAFEDEE7049B059A134317D069
:10946C0001F086F8002813D1002F11D162B6BFF39A
:10947C006F8F2000049A059B2830FEF7FDFA05003B
:10948C00EFF3108372B603936B425D41EDB2C2E70A
:10949C00236820000193009909AB07AAFFF7C2FECD
:1094AC000500B8E770B50400836908000D00984703
:1094BC000200EFF3108672B60123297820000B43CB
:1094CC002B706168FFF777FE60602000FFF73EFFAE
:1094DC00002E02D162B6BFF36F8F70BDF8B50400D9
:1094EC00EFF3108772B608212269A3680A4203D1F0
:1094FC006168CA1A8B4201D9226AD21AE169002A20
:10950C0007D1002F02D162B6BFF36F8F0026300057
:10951C00F8BD9B00CE180322CB5C03211A400B42F2
:10952C00EFD0022A02D13568AD0805D1DA0713D481
:10953C003000A36998470500A1682A002000FFF7B6
:10954C003AFE2900A0602000FFF743FE002FC7D190
:10955C0062B6BFF36F8FC3E7022213433370A36964
:10956C003000A5689847290002002000FFF723FE71
:10957C00A060002FCBD162B6BFF36F8FC7E7F8B5F1
:10958C000400836908000D0098470600EFF310876C
:10959C0072B601222B7893432B7023699B0705D558
:1095AC00E268E36992009B189D421AD102222B7843
:1095BC0093432B70A368E168994204D132002000D8
:1095CC00FFF7F9FDA06031002000FFF702FE002F2D
:1095DC0002D162B6BFF36F8F20002830FEF71AFA63
:1095EC00F8BD03222E68830016401E432E60EEE762
:1095FC0010B5EFF3108472B6036982681B0703D4AD
:10960C0041688B1A8A4201D9036A9B1A002C02D139
:10961C0062B6BFF36F8F5A1E9341D8B210BD70471C
:10962C000378020000205B070AD4136852881B03DE
:10963C005B0D1209981807231730984303308008E4
:10964C0070470020704710B5012101F0ABF810BD38
:10965C0010B501F07EF80A220023F6F717FE10BDB4
:10966C001FB502900020039103000200010001903D
:10967C000090F8F759F905B000BD10B50120F7F7C7
:10968C00CDFE10BD00207047436810B5DA71012281
:10969C004368196043685A71F7F7B0FE10BD70B596
:1096AC0006000C001500081E0ED0906853681B1A9B
:1096BC0099420AD813680A001818310001F0A0F872
:1096CC002000AB681B19AB6070BD1C204042FBE74F
:1096DC0070B50E00040015001900002802D1F7F730
:1096EC009DFE70BD002B06D013035B0D1030C0180F
:1096FC00120D01F085F8200025606660F8F724F85B
:10970C00EFE707B50123019201AAF8F73DF807BD71
:10971C0007B5009201936A460223F8F735F807BDA6
:10972C001FB50293069B0192039301AA0323F8F73A
:10973C002BF805B000BDF8B506000D0014001F0095
:10974C00002C00D1F8BD210028003A00B047241AA3
:10975C002D18F5E710B5426804000CCA8168006842
:10976C00FFF7E9FF002263681A6010BD70B54B6803
:10977C0005001A68CB680C009A4202D10800FFF76A
:10978C00E9FF6068012101F00DF8A3681D54002069
:10979C0070BD70B504000D000A2802D10D20FFF732
:1097AC00E5FF29002000FFF7E1FF002070BDF0B5B8
:1097BC008B6889B006930B880790DB0508000D7841
:1097CC000C005E0F1700F8F7FDF80023AD06010042
:1097DC006D0F984203DB2800F7F7C8FF0300210048
:1097EC00226810311203520D60888C18551EAA4144
:1097FC0052421140002200090490029107980699E8
:10980C000597039401960092F8F70AF909B0F0BD98
:10981C00436800201B685B681961704743681B68CC
:10982C001A68526853607047F7B5012143681B688A
:10983C005A6811751D686B682F681C685B68AE6888
:10984C000193002C02D16B681C60F7BD2100300025
:10985C00019AB847241A3618F3E710B543681B6809
:10986C001868F8F743FA10BD70B543680C001D6812
:10987C006B681869F7F7ACFD0F220300210028680C
:10988C00984770BD10B5FFF743FF10BD7F227023C2
:10989C0010B50240184202D0F8F75CFB10BD012154
:1098AC0043B208009040002BF8DA103291400800C7
:1098BC00F4E710B500F0ADFF10BD10B500F0A0FF3F
:1098CC0010BD10B501000068F9F7F2F910BD10B524
:1098DC00F9F74AFAF9F766FA10BD10B50021012024
:1098EC00F9F7E6F910BD10B5F9F7E2FBF9F7BAF99B
:1098FC00F9F7C4F9F9F722FCFDF76EFF8620404218
:10990C007047002802D162B6BFF36F8F7047BFF368
:10991C004F8F30BF62B6BFF36F8F704710B50B69B6
:10992C0049699847002010BD10B5F9F74BFC002091
:10993C0010BD1F23012019408840704710B513003B
:10994C000A000121FFF7E4FE10BD10B50A00012149
:10995C00FFF7D7FE10BD10B50C00F9F7ADFD0028D0
:10996C0002D08460002010BD16204042FBE710B5E9
:10997C000C00F9F7A1FD002805D0002C03D0437989
:10998C000020237010BD16204042FBE710B50400E8
:10999C00FAF794F8002802D01620404210BD20009F
:1099AC00FAF7D4F80028F9D0F6E710B5F9F784FDEA
:1099BC00002801D0008810BD16204042FBE770B58E
:1099CC007F240C402000F9F777FD010005000C31D5
:1099DC002000F9F7E9FE00232B61AB68002B02D0C5
:1099EC0001212000984770BD70B580240C432000E5
:1099FC00F9F762FD05001430FEF70CF8AB68002B8C
:109A0C0002D002212000984770BD70B503880C88E5
:109A1C009C4225D814889C4222D344884D88A54268
:109A2C001ED85588A5421BD385888C88AC4217D884
:109A3C009488AC4214D3C488CE88A64210D8D68859
:109A4C00A6420DD300890989814209D81289824224
:109A5C0006D3AB4204D80020A34200D9863870BD8F
:109A6C0086204042FBE770B504000D0086688168D3
:109A7C003031826828003A32FFF7C7FF002803D143
:109A8C00290020003369984770BD70B504000D00A3
:109A9C0083688168483182685E6C5232002E08D02F
:109AAC002800FFF7B2FF002802D129002000B047A0
:109ABC0070BD58204042FBE710B54468A469A46807
:109ACC00A04710BD10B54468A469E468A04710BD58
:109ADC0010B543689B691B69984710BD10B5FFF71B
:109AEC0010FE10BD10B513000A000121FFF710FE87
:109AFC0010BD10B5FDF7CAFE10BD10B5FDF73EFF49
:109B0C0010BDF0B50500066901225242D31710367C
:109B1C0085B03000FFF7EDFF1821280003AAFAF7F3
:109B2C000DFA041E14D10127039A18213A43280078
:109B3C000392FAF719FA041E0AD100F00AFE0090FB
:109B4C0001912800182103AAFAF7F8F9041E0CD089
:109B5C003000FFF7D2FF200005B0F0BD182128001F
:109B6C0003AAFAF7EBF900281BD1039B3B42EFD178
:109B7C0000F0EFFD009A019B801A9941002904DC4A
:109B8C00ECD1FA239B009842E8D90123039A1821BF
:109B9C009A4328000392FAF7E7F9041ED8D10B3C3C
:109BAC00D6E70400D4E7F7B50669070033790D0052
:109BBC00002B41D1103601225242D3173000FFF74F
:109BCC0098FFF023F820EC88A988013C24011C4064
:109BDC004B1E40011B0203400F201C432B882A897B
:109BEC00013B03401C43531E180401940400F8204D
:109BFC00400304402000019C9BB20443012B10D86D
:109C0C006B885B1801335A437F2A00D97F22482185
:109C1C0038001202FAF7A8F9051E08D180231B049C
:109C2C001C4322000C213800FAF79EF90500300085
:109C3C00FFF763FF2800FEBD10256D42FAE70723EE
:109C4C0000200B607047F7B506000C0015000029CA
:109C5C000BD0442101AA0769FAF770F9002807D143
:109C6C003B79002B05D104332370002D13D1002038
:109C7C00FEBD019B1A0601D50323F5E79A0601D513
:109C8C000223F1E7402219001140134201D00123B5
:109C9C00EAE72170E9E74021300001AAFAF74EF912
:109CAC000028E5D1019B2B705B045B0E6B70DEE72B
:109CBC004368DB69002901D0987B7047587BFCE72F
:109CCC0003699960DA60704737B5040005690122B1
:109CDC005242D31710352800FFF70BFF1821200034
:109CEC0001AAFAF72BF9002807D10222019B1821AF
:109CFC001A4320000192FAF737F92800FFF7FDFE0E
:109D0C0037BD40689B08406C9B00406809185B1885
:109D1C00521A994201D10020704708685050043102
:109D2C00F7E740689B08406C9B00406809185B187B
:109D3C00521A994201D100207047505801C1F8E7DE
:109D4C00436892085B6C92005B68C9180023521838
:109D5C008A4201D10020704708C1F9E7002210B5F2
:109D6C0011001520F9F77AF91520F9F75BF90022A3
:109D7C0016201100F9F772F91620F9F753F910BDF6
:109D8C007047436800205B681B690B607047436831
:109D9C005B6858694240114041405961002070474E
:109DAC00436800205B6899617047436800205B68DA
:109DBC0099627047436800205B685A695140596149
:109DCC00704710B503699868002821D088421BD1D0
:109DDC000868DC689860A14200D1D8600020086057
:109DEC00824206D09A680A60DA689960002A00D12B
:109DFC00D960002010E0814206D108682060D86844
:109E0C008142EBD1DC60E9E7040000680028F2D164
:109E1C00002AE7D11620404210BDF0B501263024AF
:109E2C0085B0029333001440019494098B40344064
:109E3C008C4040680236456803279D432C434460A0
:109E4C008468A4461C008C406643F5430395D509F1
:109E5C003D4065432F006546B5432F43876003277C
:109E6C00520A3A406243C568B5432A43C260019A1C
:109E7C00202A0CD1072914D823008B408B400F21AA
:109E8C005943026A8A4302994B4313430362019B71
:109E9C0002681B095C43039B1A401443046005B021
:109EAC00F0BD0F211B0A5B435B435943426A8A4353
:109EBC0002994B431A434262E9E71300F7B580223B
:109ECC001F00920217400C000197134220D09A07F2
:109EDC0017D55A0765D55022D90614D5802189008B
:109EEC000A43C02519008026ED002940F600B14236
:109EFC004AD0A94218D08025AD00A94217D18021A3
:109F0C0014E01022E8E79906EBD58021C900E7E7B9
:109F1C003022D903E5D5DA0603D49A06D20F920281
:109F2C00DFE780229200DCE7C02149000A43C02110
:109F3C001E0089020E40056900960B420AD02E695C
:109F4C003100E1408C46012167460F4202D1A1400D
:109F5C00314329610199002906D041681E0315D5AA
:109F6C000123A34049688B61002321004068FFF75F
:109F7C0054FF009B002B05D12B6901221900E140F5
:109F8C0011420AD10020FEBD8021CEE75B03EBD548
:109F9C000123A34049688B62E6E7A24093432B61FF
:109FAC00F0E786204042EEE770B50B0089680500AB
:109FBC00002903D05E680C68002900D170BD8B6845
:109FCC001A002A402B4202D030004B689847231EBF
:109FDC0000D0236821001C00EEE7F8B505004068AE
:109FEC001F000E001400FFF718FF112F06D10123DC
:109FFC006A68B3405268240502D593610020F8BD0D
:10A00C009362FBE730B50368136005790468ED00D3
:10A01C006419A34202D30220404230BD5C798C42C9
:10A02C0001D00833F0E70020F7E74068CB03006865
:10A03C001B0D1B181F2001401E3888401B68034055
:10A04C00591E8B410020137070474268CB03126875
:10A05C001B0D9B181F2211401E3A8A4018680243A0
:10A06C001A600020704742681F20CB0301401E3845
:10A07C00884012681B0D9B181A6882431A600020D6
:10A08C00704770B50D000400FFF7DFFF29002000BA
:10A09C00FFF7E9FF002070BD802203005201080089
:10A0AC00934207D080225205934207D14342584134
:10A0BC0001307047434258410330FAE7434258415C
:10A0CC000230F6E7012210B5436802211B68D869FB
:10A0DC00DC69C0081040144200D00843DC6904223B
:10A0EC000C4200D01043D969114201D020221043F8
:10A0FC008022D9695200114202D008211A62084309
:10A10C00C20701D508221A62820701D501221A6200
:10A11C00420701D502221A62820601D504221A6274
:10A12C0010BD802210B543681B68D8691042FCD062
:10A13C00EFF3108072B6DC69144205D10028F4D11B
:10A14C0062B6BFF36F8FF0E79962002800D010BDA4
:10A15C0062B6BFF36F8FFAE7082243681B68D869B1
:10A16C00104200D01A62DA69920603D500205B6AAD
:10A17C000B70704701204042FBE7704770B5A52576
:10A18C00AD00435D04000220012B09D0012363556F
:10A19C002068FCF741FC206800F058F9002060555D
:10A1AC0070BD70B5A525AD00435D04000220012BE8
:10A1BC0009D0012363552068FCF736FC2068FCF7B6
:10A1CC0089FE0020605570BD704770B5A525AD00A7
:10A1DC00435D04000220012B07D001236355206846
:10A1EC00617400F02DF90020605570BD70B504004D
:10A1FC0007200D000840282141436DB26618002D40
:10A20C0018DA012514316118757508700A61CB7064
:10A21C00022B01D100230B71A525AD00635D02203B
:10A22C00012B06D0012363552068FCF705FC0020A8
:10A23C00605570BD002555315636FF31FF3661181B
:10A24C003570E2E707220B000A40282151435BB22C
:10A25C0070B504004018002B12DA01231431611878
:10A26C004375A5250A70AD00635D0220012B06D055
:10A27C00012363552068FCF735FD0020605570BD47
:10A28C00002355315630FF31FF3061180370E8E779
:10A29C00F8B50724214021344C4306193700FC370C
:10A2AC003B673300002556335536FF33FF365534A4
:10A2BC007D67FA66FF341D70317001190068FCF778
:10A2CC0045FE2800F8BD07230B40282159434018B0
:10A2DC00FC30406F704770B50724214021344C434B
:10A2EC0006193500B26201223835F3622A70002556
:10A2FC003175356373637275143401190068FCF79A
:10A30C0025FE280070BD072270B5037904000A40B1
:10A31C000120934219D348B22823002816DA53435C
:10A32C00190001201431E318611858750123A52573
:10A33C008B700A70AD00625D02209A4205D06355A5
:10A34C002068FCF763FD0020605570BD4B4319007D
:10A35C000020E31855315633FF31FF336118187064
:10A36C00E4E70B000F2270B5017904001A400120BC
:10A37C0091421BD3072228211A4051435BB260182B
:10A38C00002B14DA01231431611843750025A5261E
:10A39C008D700A70B600A35D0220012B06D001233C
:10A3AC00A3552068FCF750FD2800A55570BD00236F
:10A3BC0055315630FF31FF3061180370E6E730B588
:10A3CC0028240D060BD5072529404C4314340019BD
:10A3DC0099B2002A07D10273C180002030BD4C43D2
:10A3EC005534FF34F3E7012283600273F5E710B5AF
:10A3FC0003000268B52001218000B324195000200D
:10A40C00A4001855536D194302235165516D0B432C
:10A41C00536510BD704784B010B5049201220264DC
:10A42C000593036C040093430364036C0391934002
:10A43C00D34003640020606410BC08BC04B018470F
:10A44C00002901D18023C364002070478023826DD2
:10A45C001B021343836500207047406C704710B596
:10A46C0043690400002B07D100230122E1684878DE
:10A47C0002434A70584210BD98470028F4D0C217C6
:10A48C0083185340FF2B00DDFF23E2681370ECE7C9
:10A49C00002809D00123C26800205178194202D04B
:10A4AC0010784242504118407047EFF3108372B657
:10A4BC00FEE710B5EFF3108372B6FFF728FAF9E751
:10A4CC000E2210B5825600238A4202D0FDF7CCFD35
:10A4DC000300180010BD030000209860D8601B60BA
:10A4EC005B607047002A07D08A4205D38160C26046
:10A4FC00006040600020704716204042FBE70122BC
:10A50C0030B5140003688C401D00CB40A54305609A
:10A51C001800104030BD10B5002804D000227C304B
:10A52C00110000F0CEF810BD70B50D000400102223
:10A53C00002100F06EF9656070BD13B50190080044
:10A54C00EFF3108472B601A9FDF772FB002C02D157
:10A55C0062B6BFF36F8F16BD10B5FFF7EEFF041E8A
:10A56C0004DDEFF3108072B6FDF708FE200010BD7D
:10A57C00EFF30580431E9841C0B27047582040420B
:10A58C007047002070470368426813605A600023CC
:10A59C0003604360704710B50400FFF7F4FF02221C
:10A5AC00637B934363730023A36010BD70B50400F9
:10A5BC000D00FDF7B9FC0223627B13436373002D7E
:10A5CC001CD0A5602B689D4209D16B682560636027
:10A5DC001C606C6012E06A689A42F6D01B68002B13
:10A5EC00F3D00E220E21A25659568A42F3D0914234
:10A5FC00F1DD5A682360626014605C6070BD10B558
:10A60C00EFF3108472B6FDF749FC002C02D162B650
:10A61C00BFF36F8F10BD10B5EFF3108472B6836863
:10A62C00002B01D0FFF7B7FF002C02D162B6BFF3AD
:10A63C006F8F10BD70B50400EFF3108572B6282330
:10A64C00427B1A420BD18368002B01D0FFF7A3FF8A
:10A65C000422637B200093436373FDF71FFC002DE2
:10A66C0002D162B6BFF36F8F70BD10B501211838DF
:10A67C00FFF7E0FF10BD70B5EFF3108572B60468FC
:10A68C00A0420BD0002C02D02000FFF784FF002D3D
:10A69C0002D162B6BFF36F8F200070BD0024F6E7C5
:10A6AC000200C3170021632010B580185941002304
:10A6BC006422F5F7EBFDC117FDF702FE6423584346
:10A6CC0010BD030070B5EFF3108572B6046800205E
:10A6DC00A3420ED084420CD0E16622612000FFF729
:10A6EC005AFF2000183000F00AF82000FDF7D6FBC6
:10A6FC000120002D02D162B6BFF36F8F70BD70B513
:10A70C000400EFF3108572B60368002B1AD0FDF726
:10A71C0081FF06002000FDF7ADFF802300221B0601
:10A72C0022616361A64206D1FDF798FFFDF77AFF1F
:10A73C000021FBF713FB0020002D02D162B6BFF302
:10A74C006F8F70BD16204042F6E710B5FEF7A8F8E3
:10A75C0010BD10B5FEF7A4F810BD42620200002334
:10A76C001832016203638261C26103604360436318
:10A77C00704710B50400FFF7C2FF002811D1636ABF
:10A78C00002B01D02000984720001830FFF773FFF2
:10A79C00002806D0FFF733FFEFF3108072B6FDF7F9
:10A7AC00EDFC10BD0300EFF3108272B60068411887
:10A7BC001960002A02D162B6BFF36F8F7047030095
:10A7CC00EFF3108272B60068411A1960002A02D1A8
:10A7DC0062B6BFF36F8F70470300EFF3108272B64F
:10A7EC0000681960002A02D162B6BFF36F8F704700
:10A7FC00030010B50C33C3600361FEF715FC10BDEC
:10A80C00002310B59A4200D110BDCC5CC454013366
:10A81C00F8E703008218934200D170471970013396
:10A82C00F9E730B50500101E0BD00024013A2B5D62
:10A83C00085D834204D1A24202D00134002BF6D130
:10A84C00181A30BD030041188B4202D01A78002A26
:10A85C0001D1181A70470133F6E7F0B50D00372116
:10A86C00C91A8FB0C9B20D911F2104000B400C9373
:10A87C000C99E3B2082955D0102900D164E0E907FE
:10A88C0060080843690806900791A008A9070843C7
:10A89C00A90808900991089E099F069807998019A4
:10A8AC0079410E07B446060900966646009F374369
:10A8BC000E0900970196009E019F801979410E06A2
:10A8CC00B4466746060A3E4302960E0A0396029E5B
:10A8DC00039F801979410E04B4466746060C3E432B
:10A8EC0004960E0C0596049E059F8019794100264E
:10A8FC000A910B960A9E0B9F801979414E07CD0841
:10A90C000521C4083443614349005B1ADBB2092BAF
:10A91C0012D9012000210A3B24184D41DBB21DE065
:10A92C000200A5E707210B4069078C466646E00844
:10A93C00E908064334000D00303313702300501C1B
:10A94C002B43EDD10FB0F0BD0F210B4029078C46E6
:10A95C00664620092909064334000D00092BEBD962
:10A96C000D99CB18DBB2E7E70B694A69934202D029
:10A97C005A1C0A6118707047014800687047000043
:04A98C00200A00207D
:08A99000AE59FF7F0100000039
:10A998000000000030AA00080112000800000000B2
:10A9A800658A0008000000000000000050AA0008A6
:10A9B8000000000030AB00080000000010AB0008E9
:10A9C8000000000070AA000800000000D0AA0008DB
:10A9D8000000000090AA000800000000F0AA00088B
:10A9E80000000000B0AA000865320008000000005E
:10A9F8000000000050AB00082154000800000000CF
:10AA0800D15C000800000000E1120008000000000E
:10AA1800F931000800000000D17A000800000000A9
:08AA28000000000070AB000803
:10AA300017C500080000000018AD000854000020F1
:10AA4000000000003152000800000000000000007B
:10AA500078C5000874B0000808AD00086200002046
:10AA600000000000000000000000000000000000E6
:10AA7000C6BB0008000000000000000050000020DD
:10AA800000000000E93300080000000000000000A2
:10AA900024C5000894AF0008E4AC0008560000206C
:10AAA0006013002025550008000000000000000091
:10AAB00032C50008A8AF0008E4AC00085800002028
:10AAC000741300202555000800000000000000005D
:10AAD00040C50008BCAF0008E4AC00085A000020E4
:10AAE0008813002025550008000000000000000029
:10AAF0004EC50008D0AF0008E4AC00085C000020A0
:10AB00009C130020255500080000000000000000F4
:10AB10005CC50008E4AF0008E4AC00085E0000205B
:10AB2000B0130020255500080000000000000000C0
:10AB30006AC50008F8AF0008E4AC00086000002017
:10AB4000C41300202555000800000000000000008C
:10AB50002BC6000878B0000834AD0008640000205F
:10AB600020000020E1580008000000000000000064
:10AB7000FEC40008DCAE000888AC000852000020CB
:10AB8000DC110020D14E0008000000000000000091
:10AB900000000000E798000800000000E7980008A7
:10ABA00000000000E798000800000000E798000897
:10ABB00000000000E79800088EBB00081D32000866
:10ABC0008CBB00081D3200088ABB00081D3200083B
:10ABD00000000000F134000800000000E7980008C1
:10ABE00000000000E798000800000000E798000857
:10ABF00000000000E798000800000000E798000847
:10AC000000000000E798000800000000E798000836
:10AC100000000000E798000800000000E798000826
:10AC200000000000E798000800000000E798000816
:10AC300000000000E798000870AB000841440008DD
:10AC400070AB0008B543000800000000E79800085A
:10AC500000000000E798000800000000E7980008E6
:10AC600000000000E798000800000000E7980008D6
:10AC700000000000E798000800000000E7980008C6
:08AC800000000000E798000845
:10AC88004B9C0008F1410008954A0008ED42000875
:10AC98008D410008F1450008DD480008F149000829
:10ACA800539C0008CD9C0008E94F0008BD9C000893
:10ACB8000100000002000200010080000000000105
:10ACC80080000002B39B00080100000001000100A1
:0CACD8000100100000002000100020000F
:10ACE400C79E00088F9D00089B9D0008AD9D00082D
:10ACF400B79D0008C19D000875540008CF9D000849
:04AD0400000000004B
:10AD080037A0000857A0000873A000088FA000080B
:10AD180081500008C150000800000000F1500008F0
:0CAD2800FD51000800000000A5510008CB
:10AD340065A100082FA10008D1A00008015B00084C
:0CAD44002956000800000000000000007C
:10AD50004DBF00080300000034C4000803000000D9
:10AD60000BC5000803000000B8B500080300000090
:10AD700022B3000804000000E4BB00080300000048
:10AD800083BB00080300000062B400080400000058
:10AD9000E5B5000803000000E9B500080300000065
:10ADA0000EB7000803000000D8B50008040000003A
:10ADB00016C7000803000000B9B300080400000033
:10ADC000C6BE000803000000C9B50008030000006B
:10ADD0003BC6000803000000BFBE000803000000DF
:10ADE000FDB9000803000000DCB800080300000003
:10ADF0000AB500080400000029BA0008030000009A
:10AE000090AE000808000020FDB600080100000018
:10AE100001000600070002000600000010AB000859
:10AE20000200000030AB000808000000C001002054
:10AE300000010000879600082D960008020000001F
:10AE4000BB970008000000000000000000000000A8
:10AE500000000000DDB60008E5B6000800000000B4
:10AE60000000000000000000EDB60008F1B6000888
:10AE7000F5B60008F9B6000880AE000830080020DA
:10AE8000851D00084808002058140020010000001B
:10AE900075980008679800083598000829980008F8
:10AEA000000000001D98000800000000B4AE00087B
:10AEB00001000000BCAE00080200000070010000AC
:10AEC0000000000090010000000000003C000000B5
:10AED000002000000500000058002C0000000000C9
:10AEE0000000000000127A0048E8010000000000A5
:10AEF00040420F0080AF000850AF000800001C0067
:10AF0000080003000300000003000300000000002D
:10AF10007000B000880160026002780250030000F7
:10AF200024AF00080068004050B700400200000055
:10AF300040AF0008699D000860AF000800000000F5
:10AF40003C000000001000000B0000005800280129
:10AF5000481300206812002028120020031C08005B
:10AF600068AF00080100000070AF00080200000098
:10AF700003020000000000002302000000000000A7
:10AF8000B94D0008454E00080F9D00082F9D000890
:10AF90004D9D0008FFFF0000001400500500000058
:10AFA0003400000020000000FFFF000000100050EF
:10AFB000040000003400000010000000FFFF00004B
:10AFC000000C0050030000003400000008000000E6
:10AFD000FFFF0000000800500200000034000000E5
:10AFE00004000000FFFF000000040050010000000A
:10AFF0003400000002000000FFFF000000000050CD
:10B0000000000000340000000100000030AB000828
:10B0100010AB0008F0AA0008D0AA0008B0AA0008E7
:10B0200090AA0008000000000000000000000000DE
:10B030000000000000000000000000000000000010
:10B040000000000000000000000000000000000000
:10B0500000000000000000000000000000000000F0
:10B0600000000000000000000000000000000000E0
:10B0700000000000001002400038014050AA000803
:10B080000E0600009CB00008010000000000000057
:10B090000000000000000000A4B000084000000014
:10B0A00000400000ACB0000801000000B4B000088F
:10B0B000020000008104000000020000A104000062
:10B0C0000000000000000000000000000000000080
:10B0D0000000000000000000000000000000000070
:10B0E000000000000100000002000000030000005A
:10B0F0000400000006000000070000000800000037
:10B1000009000000CCC60008DAC60008EEC6000838
:10B11000FDC6000809C7000898A9000898A90008FA
:10B1200008AA000810AA000830AA000830AA0008DF
:10B1300019C7000800010000000000000010000016
:10B1400000304557532043414E204644204344435A
:10B1500020436F6D706F73697465204669726D77F7
:10B16000617265207374617274696E672E2E2E0091
:10B17000537461747573204C45442064657669632B
:10B1800065206E6F74207265616479004572726F1C
:10B190007220636F6E6669677572696E672073747B
:10B1A00061747573204C45443A20256400466169FA
:10B1B0006C656420746F20696E697469616C697A6A
:10B1C00065205046455420636F6E74726F6C3A2050
:10B1D0002564004661696C656420746F20696E693E
:10B1E0007469616C697A65205553422067735F7595
:10B1F00073623A202564004661696C656420746F4F
:10B2000020696E697469616C697A652043444320E2
:10B2100068616E646C65723A202564004661696CF1
:10B22000656420746F20696E697469616C697A6500
:10B230002067735F7573622043414E3A2025640096
:10B24000455753206669726D7761726520696E6932
:10B250007469616C697A656420737563636573737F
:10B2600066756C6C79004344432041434D2064650E
:10B2700076696365206E6F7420726561647900433E
:10B2800044432068616E646C657220696E697469FC
:10B29000616C697A65640050464554315F4F4E00D9
:10B2A0005046455431204F4E0D0A0050464554310A
:10B2B0005F4F4646005046455431204F46460D0AE2
:10B2C0000050464554325F4F4E00504645543220A0
:10B2D0004F4E0D0A0050464554325F4F46460050CF
:10B2E00046455432204F46460D0A005354415455AA
:10B2F000530050464554313A2025732C2050464582
:10B3000054323A2025730D0A004552524F523A20CA
:10B31000556E6B6E6F776E20636F6D6D616E640D31
:10B320000A006364635F68616E646C657200504616
:10B330004554204750494F20646576696365732002
:10B340006E6F74207265616479004661696C656432
:10B3500020746F20636F6E66696775726520504652
:10B360004554312070696E3A202564004661696C4D
:10B37000656420746F20636F6E66696775726520FF
:10B3800050464554322070696E3A2025640050467C
:10B39000455420636F6E74726F6C20696E697469B6
:10B3A000616C697A6564005046455431202573000C
:10B3B000504645543220257300706665745F636F94
:10B3C0006E74726F6C0025733A2052583A204944CB
:10B3D0003D30782530387820444C433D2564004387
:10B3E000414E20646576696365206E6F74207265D6
:10B3F000616479004661696C656420746F207365CF
:10B40000742043414E2074696D696E673A2025644B
:10B41000004661696C656420746F20616464204338
:10B42000414E2052582066696C7465723A2025643A
:10B430000067735F7573622043414E20696E7465C7
:10B44000726661636520696E697469616C697A65A9
:10B45000640063616E5F72785F63616C6C626163EC
:10B460006B0067735F7573625F63616E0025733A8B
:10B4700020576F756C642073656E642025642062AC
:10B480007974657320746F20686F737400496E69F6
:10B490007469616C697A696E67206D696E696D6146
:10B4A0006C2067735F7573622055534220696E7418
:10B4B000657266616365004661696C656420746FDE
:10B4C00020656E61626C65205553423A2025640008
:10B4D00042617369632055534220696E74657266D8
:10B4E00061636520696E697469616C697A6564007D
:10B4F00067735F7573625F73656E645F6672616DBB
:10B50000655F746F5F686F7374007573625F6773F4
:10B510005F7573620028756E7369676E65642920B4
:10B5200063686172202A207573656420666F7220DB
:10B5300025257020617267756D656E742E204974C3
:10B540002773207265636F6D6D656E64656420742A
:10B550006F206361737420697420746F20766F6943
:10B5600064202A2062656361757365206974206DAB
:10B570006179206361757365206D697362656861C7
:10B5800076696F7220696E206365727461696E20DE
:10B59000636F6E66696775726174696F6E732E2072
:10B5A000537472696E673A2225732220617267753F
:10B5B0006D656E743A25640063627072696E7466BC
:10B5C0005F7061636B6167650073746D33325F62D6
:10B5D00061636B75705F646F6D61696E006C6F673E
:10B5E00067696E67006C6F67006C6F675F6D676D92
:10B5F00074004D65737361676520282225732229C5
:10B600002064726F70706564206265636175736534
:10B6100020697420657863656564732073697A6551
:10B62000206C696D69746174696F6E2028257529B5
:10B63000004D6573736167652064726F7070656437
:10B640002062656361757365206974206578636540
:10B650006564732073697A65206C696D69746174BF
:10B66000696F6E2028257529001B5B306D002573DE
:10B6700020005B2530386C755D20005B253032750D
:10B680003A253032753A253032752E253033752CF7
:10B69000253033755D200025732F003C25733E2037
:10B6A0000025733A20002530327820002020200029
:10B6B0007C00256300206D6573736167657320648A
:10B6C000726F70706564202D2D2D0D0A1B5B306D1F
:10B6D000001B5B313B33316D2D2D2D20001B5B3169
:10B6E0003B33316D001B5B313B33336D0065727250
:10B6F0000077726E00696E6600646267006C6F6747
:10B700005F6261636B656E645F75617274006C6F1C
:10B71000675F75617274005365742068616C742092
:10B7200065702030782530327800436C6561722076
:10B7300068616C742065702030782530327800455F
:10B740006E64706F696E74203078253032782069AD
:10B750007320696E76616C696400456E64706F6910
:10B760006E742030782530327820616C72656164A7
:10B77000792064697361626C6564004661696C6517
:10B780006420746F2064697361626C6520656E6407
:10B79000706F696E742030782530327800456E64A1
:10B7A000706F696E742030782530327820616C7249
:10B7B0006561647920636F6E6669677572656400A0
:10B7C0004661696C656420746F20636F6E6669679B
:10B7D00075726520656E64706F696E7420307825AF
:10B7E00030327800456E64706F696E742030782551
:10B7F00030327820616C726561647920656E6162B7
:10B800006C6564004661696C656420746F20656EC8
:10B8100061626C6520656E64706F696E742030784B
:10B8200025303278004661696C656420746F20773A
:10B830007269746520656E64706F696E74206275DC
:10B8400066666572203078253032780052657175F1
:10B850006573742062756666657220746F6F2073FD
:10B860006D616C6C00555342206465766963652098
:10B87000737570706F727420616C72656164792089
:10B88000656E61626C6564004661696C6564207414
:10B890006F20636F6E66696775726520555342202D
:10B8A00064657669636520737461636B00457272C9
:10B8B0006F6E656F75732064657669636520646576
:10B8C0007363726970746F72206F7220624D617859
:10B8D0005061636B657453697A6530007573625F9C
:10B8E0006465766963650030313233343536373814
:10B8F0003941424344454600546865726520697386
:10B90000206E6F207573625F6366675F6461746148
:10B9100020666F7220257000556E696E69746961CA
:10B920006C697A6564207573625F6366675F6461E2
:10B93000746120706F696E7465722C20636F72720F
:10B9400075707465642064657669636520646573E9
:10B9500063726970746F723F004661696C65642040
:10B96000746F2076616C696461746520656E6470C3
:10B970006F696E747300746865206E657720534E2E
:10B980002064657363726970746F7220646F65738D
:10B990006E27742068617665207468652073616D18
:10B9A00065206C656E67746820617320434F4E4656
:10B9B00049475F5553425F4445564943455F534E9F
:10B9C00000496E636F6D706C65746520646576699F
:10B9D00063652064657363726970746F7200466199
:10B9E000696C656420746F206669787570205553A2
:10B9F000422064657363726970746F72007573625C
:10BA00005F64657363726970746F72005472616E03
:10BA100073666572206572726F722025642C2065D2
:10BA20007020307825303278007573625F747261EF
:10BA30006E736665720072302F61313A2020307863
:10BA400025303878202072312F61323A202030782A
:10BA500025303878202072322F61333A2020307818
:10BA6000253038780072332F61343A202030782521
:10BA7000303878207231322F69703A2020307825A2
:10BA8000303878207231342F6C723A20203078258B
:10BA90003038780020787073723A20203078253062
:10BAA0003878004661756C74696E6720696E7374CE
:10BAB00072756374696F6E2061646472657373205C
:10BAC000287231352F7063293A2030782530387844
:10BAD00000556E68616E646C6564204952516E3A1F
:10BAE000202564005265736572766564204578632D
:10BAF000657074696F6E20280053707572696F7578
:10BB00007320696E74657272757074202849525181
:10BB10002000535053454C20696E20746872656153
:10BB200064206D6F646520646F6573206E6F742090
:10BB3000696E64696361746520505350002A2A2A33
:10BB40002A2A2048415244204641554C54202A2A52
:10BB50002A2A2A00415243485F4558434550542001
:10BB60007769746820726561736F6E2025780A00AA
:10BB70002A2A2A2A2A20257320256429202A2A2ACB
:10BB80002A2A006765746F707400040C02020002B8
:10BB9000436C6F636B20636F6E74726F6C206465AF
:10BBA00076696365206E6F742072656164790049FF
:10BBB0006E76616C6964206C696E65206E756D626D
:10BBC000657220257500696E746572727570742DCA
:10BBD000636F6E74726F6C6C6572403430303231EA
:10BBE00038303000657874695F73746D3332004E9D
:10BBF0006F742076616C696420656E64706F696E25
:10BC0000743A202530327800696E76616C69642060
:10BC100065702030782530327800636C6F636B205C
:10BC2000636F6E74726F6C20646576696365206EF5
:10BC30006F7420726561647900436F756C64206E67
:10BC40006F742073656C6563742055534220646F74
:10BC50006D61696E20636C6F636B00556E61626C21
:10BC60006520746F20656E61626C652055534220BB
:10BC7000636C6F636B004661696C656420746F2050
:10BC80006765742055534220646F6D61696E20634F
:10BC90006C6F636B20726174650055534220436C76
:10BCA0006F636B206973206E6F742034384D487A4F
:10BCB0002028256429005553422070696E637472F0
:10BCC0006C207365747570206661696C65642028EA
:10BCD000256429005043445F496E69742066616998
:10BCE0006C65642C202564005043445F53746F706E
:10BCF000206661696C65642C202564005043445FB4
:10BD00005374617274206661696C65642C202564CB
:10BD10000048414C5F5043445F5365744164647212
:10BD2000657373206661696C6564283078253032EC
:10BD300078292C2025640048414C5F5043445F45DE
:10BD4000505F52656365697665206661696C6564FC
:10BD500028307825303278292C20256400696E76C9
:10BD6000616C696420656E64706F696E7420636FC6
:10BD70006E66696775726174696F6E00656E647076
:10BD80006F696E7420696E6465782F616464726592
:10BD90007373206F7574206F662072616E67650023
:10BDA00048414C5F5043445F45505F536574537442
:10BDB000616C6C206661696C65642830782530326E
:10BDC00078292C2025640048414C5F5043445F454E
:10BDD000505F436C725374616C6C206661696C6572
:10BDE0006428307825303278292C20256400484199
:10BDF0004C5F5043445F45505F4F70656E206661F5
:10BE0000696C656428307825303278292C202564C7
:10BE10000048414C5F5043445F45505F436C6F7333
:10BE200065206661696C6564283078253032782930
:10BE30002C20256400556E61626C6520746F20674C
:10BE40006574207772697465206C6F636B20282598
:10BE500064290048414C5F5043445F45505F547231
:10BE6000616E736D6974206661696C6564283078F1
:10BE700025303278292C20256400496E76616C6962
:10BE80006420456E64706F696E7420257800577267
:10BE90006F6E6720656E64706F696E74206469727E
:10BEA000656374696F6E3A203078253032780057B8
:10BEB000726F6E6720617267756D656E7473007561
:10BEC00073625F64635F73746D33320065787465A9
:10BED0006E646564007374616E6461726400696E9F
:10BEE00076616C6964206672616D6520776974683B
:10BEF000202573202825642D626974292043414E32
:10BF000020494420307825302A7800696E76616CAB
:10BF100069642066696C746572207769746820258D
:10BF200073202825642D626974292043414E2049DD
:10BF30004420307825302A782C2043414E20494433
:10BF4000206D61736B20307825302A780063616E34
:10BF50005F636F6D6D6F6E006661696C6564207400
:10BF60006F207265616420726567203078253033F8
:10BF700078202865727220256429006661696C65E5
:10BF80006420746F20777269746520726567203051
:10BF90007825303378202865727220256429006660
:10BFA00061696C656420746F2072656164205278E9
:10BFB000204649464F206865616465722028657295
:10BFC0007220256429006661696C656420746F20A5
:10BFD00072656164205278204649464F206461743E
:10BFE00061202865727220256429004672616D65A2
:10BFF00020697320746F6F20626967006661696CE5
:10C00000656420746F20656E61626C652043414EEB
:10C01000207472616E73636569766572202865723B
:10C020007220256429006661696C656420746F2044
:10C030006C6561766520696E6974206D6F6465203A
:10C04000286572722025642900756E737570706F93
:10C0500072746564206D6F64653A203078253038DD
:10C0600078004D657373616765206C6F7374206F22
:10C070006E204649464F30004D65737361676520F9
:10C080006C6F7374206F6E204649464F31006661B5
:10C09000696C656420746F20726561642074782017
:10C0A0006576656E74206669666F202865727220F9
:10C0B000256429005458204649464F20656C656D1B
:10C0C000656E74206C6F73740041636365737320D5
:10C0D000746F207265736572766564206164647242
:10C0E000657373004D6573736167652052414D2020
:10C0F000616363657373206661696C757265007551
:10C100006E737570706F727465642043414E206663
:10C1100072616D6520666C616773203078253032FE
:10C12000780043414E20464420666F726D61742052
:10C130006E6F7420737570706F7274656420696EB1
:10C14000206E6F6E2D4644206D6F646500646174CF
:10C1500061206C656E6774682028257A7529203EF9
:10C16000206D6178206672616D6520646174612064
:10C170006C656E6774682028257A752900444C43E5
:10C18000206F6620256420666F722043414E204652
:10C190004420666F726D6174206672616D65004443
:10C1A0004C43206F6620256420666F72206E6F6E90
:10C1B0002D464420666F726D6174206672616D65F4
:10C1C000006661696C656420746F207772697465BC
:10C1D00020547820427566666572206865616465E2
:10C1E00072202865727220256429006661696C6579
:10C1F0006420746F207772697465205478204275CA
:10C2000066666572206461746120286572722025FB
:10C210006429006661696C656420746F20777269B7
:10C220007465207374642066696C74657220656C33
:10C23000656D656E74202865727220256429004E34
:10C240006F2066726565207374616E64617264202C
:10C2500069642066696C746572206C65667400752B
:10C260006E737570706F727465642043414E206602
:10C27000696C74657220666C616773203078253054
:10C280003278004E6F206672656520657874656E41
:10C290006465642069642066696C746572206C65ED
:10C2A00066740066696C74657220494420256420B8
:10C2B0006F7574206F6620626F756E6473006661BF
:10C2C000696C656420746F20636C656172206578A9
:10C2D000742066696C74657220656C656D656E743A
:10C2E000202865727220256429006661696C656486
:10C2F00020746F20636C65617220737464206669BA
:10C300006C74657220656C656D656E74202865724D
:10C310007220256429004661696C656420746F2071
:10C32000656E74657220696E6974206D6F64650056
:10C330006661696C656420746F2064697361626C06
:10C34000652043414E207472616E73636569766542
:10C3500072202865727220256429004661696C6527
:10C360006420746F206578697420736C6565702033
:10C370006D6F64650043414E207472616E73636536
:10C3800069766572206E6F7420726561647900430E
:10C39000616E27742066696E642074696D696E67CA
:10C3A00020666F7220676976656E20706172616DBC
:10C3B0000043616E27742066696E642074696D693C
:10C3C0006E6720666F7220676976656E206461749F
:10C3D00061706861736520706172616D006661698A
:10C3E0006C656420746F207365742074696D696E68
:10C3F00067202865727220256429006661696C6572
:10C400006420746F207365742064617461207068A7
:10C410006173652074696D696E672028657272208A
:10C42000256429000001020304050607080C101406
:10C430001820304063616E5F6D63616E0043414E52
:10C440002070696E6374726C2073657475702066F9
:10C4500061696C6564202825642900436F756C64EC
:10C46000206E6F742073656C6563742063616E5F0A
:10C4700073746D3332666420646F6D61696E20631E
:10C480006C6F636B00436F756C64206E6F74207407
:10C4900075726E206F6E2043414E20636C6F636B2C
:10C4A0002028256429004661696C65642063616CFD
:10C4B0006C20636C6F636B5F636F6E74726F6C5F25
:10C4C0006765745F726174652870636C6B5B315D66
:10C4D00029004661696C65642063616C6C20636C43
:10C4E0006F636B5F636F6E74726F6C5F6765745FB1
:10C4F000726174652870636C6B5B305D29006361E9
:10C500006E4034303030363830300063616E5F73E7
:10C51000746D33326664007263634034303032319C
:10C52000303030006770696F403530303031343032
:10C5300030006770696F4035303030313030300056
:10C540006770696F4035303030306330300067706D
:10C55000696F403530303030383030006770696F87
:10C56000403530303030343030006770696F4035DE
:10C57000303030303030300072657365742D636F49
:10C580006E74726F6C6C6572004661696C656420D4
:10C5900063616C6C20636C6F636B5F636F6E74724E
:10C5A0006F6C5F6765745F726174652870636C6B34
:10C5B000656E5B305D2900556E61626C6520746F3D
:10C5C0002073657420257320746F20256400436FE9
:10C5D000756C64206E6F7420656E61626C652028D6
:10C5E0004C50295541525420636C6F636B00726547
:10C5F00073657420636F6E74726F6C6C6572206EFD
:10C600006F7420726561647900257320646F6573AF
:10C61000206E6F7420737570706F7274206472690D
:10C6200076657220656E61626C6500736572696122
:10C630006C40343030313338303000756172745FA3
:10C6400073746D33320048616C74696E672073795E
:10C650007374656D00556E6B6E6F776E20657272C8
:10C660006F7200756E6B6E6F776E003E3E3E205AA5
:10C67000455048595220464154414C204552524F52
:10C68000522025643A202573206F6E204350552098
:10C690002564004661756C7420647572696E67204C
:10C6A000696E746572727570742068616E646C690D
:10C6B0006E670A0043757272656E742074687265E5
:10C6C00061643A20257020282573290043505520A5
:10C6D000657863657074696F6E00556E68616E642D
:10C6E0006C656420696E7465727275707400537441
:10C6F00061636B206F766572666C6F77004B657255
:10C700006E656C206F6F7073004B65726E656C2088
:10C7100070616E6963006F7300737973776F726B0A
:10C7200071002A2A2A20426F6F74696E67205A6549
:10C7300070687972204F53206275696C642076347A
:10C740002E332E30202A2A2A0A00286E756C6C2976
:0CC75000002A666C6F61742A0000000073
:10C75C005B9100084F96000878AE000800000000BE
:10C76C0000000000359900080000000000000000E7
:10C77C00000000002800002000C20100000103009E
:10C78C000024F400C800000038000020380000200D
:10C79C00FFFFFFFFFFFFFFFFFFFFFFFFFFFFFFFF9D
:10C7AC00000000000000000000000000000000007D
:08C7BC00000000000000000075
:10C7C4000000000000000000000000000000000065
:10C7D4000000000000000000000000000000000055
:10C7E4000000000000000000000000000000000045
:08C7F40000000000000000003D
:04C7FC000000000039
:10C800000000000070340020002000000000000044
:04C810000000000024
:10C81400B8000020B8000020000000000000000064
:04C824000E00000002
:10C82800CC000020CC000020000000000100000027
:10C838001201000200000040501D6F600304010255
:10C84800030109020000000100E0320403090408A2
:10C858000345575300000024034557532067735F6F
:10C868007573622043414E2D4644000000000000CD
:10C8780000000000000000000000002203303132F8
:10C888003334353637383941424344454600000091
:0FC8980000000000000000000000000000000091
:04C8A80015E015E0A2
:0400000508002F2D93
:00000001FF
